:100000000C9463000C948B000C948B000C948B006C
:100010000C948B000C94F91C0C948B000C948B00AA
:100020000C948B000C948B000C948B000C948B0024
:100030000C948B000C948B000C948B000C948B0014
:100040000C94901B0C948B000C945E1B0C94381B2E
:100050000C948B000C948B000C948B000C948B00F4
:100060000C94DA1B0C948B00000000002400270085
:100070002A0000000000250028002B0000000000DE
:1000800023002600290004040404040404040202DA
:100090000202020203030303030301020408102007
:1000A0004080010204081020010204081020000012
:1000B0000008000201000003040700000000000027
:1000C0000000741DCA3011241FBECFEFD8E0DEBF80
:1000D000CDBF27E0AAECB4E001C01D92AD32B2075B
:1000E000E1F714E0A0E0B1E0EAEFFFE602C005901E
:1000F0000D92AA3CB107D9F710E0C2E6D0E004C0E7
:100100002197FE010E94EF35C136D107C9F70E9441
:100110005E1E0C94F0370C940000982F2091E4059B
:1001200081E0213208F043C08091C0058111FCCFED
:100130008091E30532E03093C0059093BF059FEFB7
:100140009093BE051092BD052093BC05A3ECB5E0CD
:10015000ECE9F5E090E0291331C010929B059091F5
:100160009B05880F892B80939B0580919A05813090
:1001700049F510929A0580919B058093BB00809170
:10018000BC0083FDF8CF85EC8093BC008091C00556
:100190008230E1F38091BE058F3FB1F08091BE05C2
:1001A0008032A1F08091BE05803391F084E01092FE
:1001B000C2051092E4051092C10508953D91319356
:1001C0009F5FC9CF85EEE0CF80E0F1CF82E0EFCF37
:1001D00083E0EDCF8091780590917905891B990B8B
:1001E0000895089508952F923F924F925F926F92D3
:1001F0007F928F929F92AF92BF92CF92DF92EF92B7
:10020000FF920F931F93CF93DF93CDB7DEB76C9719
:100210000FB6F894DEBF0FBECDBF522E3D874E877E
:10022000252E462E372E782E692EA982BF86C88AA3
:10023000D98AEA8AFB8A0C8B1D8B988E8F8A2115AE
:1002400000EA30070CEA400709EB500703E06007BB
:1002500071058105910509F098F52F3F10EE3107E2
:1002600015EF410715E051076105710581059105FD
:1002700009F008F40BC12F3F354D41415E47634003
:1002800071058105910509F008F40BC129813F85AD
:10029000488959896A897B898C899D89A0E099243C
:1002A00093940E94CF35C9F4F1E0FE8B04E0802ED8
:1002B000912CA12CB12C89869A86AB86BC8616C15E
:1002C000512CB0EABD87ECEAEE8789EB282E93E04B
:1002D000492E312C712C612CD9CFA52CBD84CE8414
:1002E000D22CE42CF32C072D162D29813F8548892B
:1002F00059896A897B898C899D890E941A35298749
:100300003A874B875C8729853A854B855C85B6E0C3
:10031000AB2EB12C263031054105510568F0898599
:100320009A85AB85BC8589309740A105B105E0F081
:10033000F8E0AF2EA7E0BA2EC12CD12CE12CF12C85
:1003400000E010E029813F85488959896A897B89C5
:100350008C899D890E941A35522E3D874E87252E05
:10036000462E372E782E692EA52CBD84CE84D22C15
:10037000E42CF32C072D162D29813F8548895989B6
:100380006A897B898C899D890E941835AA24AA9440
:10039000BB24BA94EFE0CE2ED12CE12CF12C00E05E
:1003A00010E00E945534A52CBD84CE84D22CE42CC0
:1003B000F32C072D162D0E941A35A32FF42FE52FAD
:1003C000422F5A2F6F2F7E2FCC24CA94DC2C8FE023
:1003D000E82EF12C411551056105710521F4C12C60
:1003E000D12C7601C394AA24A3949A1409F4E5C0ED
:1003F00001E00E8BCB01BA0137E0660F771F881F33
:10040000991F3A95D1F7A70196010E941434298FBC
:100410003A8F4B8F5C8F89849A84AB84BC8447E08D
:10042000880C991CAA1CBB1C4A95D1F79501840124
:1004300012502109310948015901298D3A8D4B8DFE
:100440005C8D280D391D4A1D5B1DAF89B88D2D931C
:100450003D934D935C931397FD016483758386836D
:1004600097831896CD92DD92ED92FC921B978E8821
:10047000882009F481C059829D849F86AE84A88A11
:10048000298A4A8A3B8A7C8A6D8A76C0512C01EE81
:100490000D8715EF1E8725E0222E412C312C712C63
:1004A000612C29813F85488959896A897B898C8992
:1004B0009D89A0E0912C0E94CF3509F00ECFA52C8C
:1004C000BD84CE84D22CE42CF32C072D162D20E0F5
:1004D00034E04BE654EF64E170E080E090E00E948D
:1004E0001A3529873A874B875C871E8A89849A84C4
:1004F000AB84BC84A501940160E070E0CB01A52C25
:10050000BD84CE84D22CE42CF32C072D162D298308
:100510003A834B835C836D837E838F83988760E00F
:1005200070E080E090E00E94553429833F87488B3B
:10053000598B6A8B7B8B8C8B9D8B0E89C12CD12C1C
:100540007601C39440E050E0BA01013009F052CF87
:10055000AF89B88D1D921D921D921C921397FD01BB
:10056000148215821682178281E090E0A0E0B0E04C
:1005700080879187A287B38729813F8548895989D8
:100580006A897B898C899D896C960FB6F894DEBF49
:100590000FBECDBFDF91CF911F910F91FF90EF90D4
:1005A000DF90CF90BF90AF909F908F907F906F9093
:1005B0005F904F903F902F900895AF89B88D1D9216
:1005C0001D921D921C921397FD01148215821682B2
:1005D000178281E090E0A0E0B0E080879187A28759
:1005E000B3875982FD85FF878E84888A49CFDF9241
:1005F000EF92FF920F931F93CF93DF93FC01E08064
:10060000F18002811381D481C581B681D7809701A1
:10061000A8016D2F7C2F8B2F9D2D35534C405109F8
:1006200061097109810991092F3F34434C405105FB
:10063000610571058105910509F0D0F49701A801C4
:100640006D2F7C2F8B2F9D2D07E00E9487352083F7
:10065000318342835383648375838683978387E0E2
:10066000DF91CF911F910F91FF90EF90DF90089550
:100670009701A8016D2F7C2F8B2F9D2D3A56484155
:10068000510961097109810991092F3F3946484192
:100690005105610571058105910509F098F49701EF
:1006A000A8016D2F7C2F8B2F9D2D06E00E94873592
:1006B0002083318342835383648375838683978346
:1006C00086E0CECF9701A8016D2F7C2F8B2F9D2D1B
:1006D000345D4043510961097109810991092F3F36
:1006E000334D40435105610571058105910509F0C0
:1006F00098F49701A8016D2F7C2F8B2F9D2D05E07D
:100700000E948735208331834283538364837583BA
:100710008683978385E0A4CF9701A8016D2F7C2F56
:100720008B2F9D2D385A4146510961097109810964
:1007300091092F3F374A41465105610571058105F1
:10074000910509F098F49701A8016D2F7C2F8B2F4C
:100750009D2D04E00E94873520833183428353839B
:10076000648375838683978384E07ACF9701A80199
:100770006D2F7C2F8B2F9D2D3055434C51096109D6
:100780007109810991092F3F3F44434C510561058F
:1007900071058105910509F098F49701A8016D2F65
:1007A0007C2F8B2F9D2D03E00E9487352083318382
:1007B00042835383648375838683978383E050CF1A
:1007C0009701A8016D2F7C2F8B2F9D2D305A464805
:1007D000514061097109810991092F3F3F494648FC
:1007E0005140610571058105910509F098F4970163
:1007F000A8016D2F7C2F8B2F9D2D02E00E94873545
:1008000020833183428353836483758386839783F4
:1008100082E026CF9701A8016D2F7C2F8B2F9D2D75
:1008200030544D40534061097109810991092F3FAE
:100830003F434D405340610571058105910509F025
:1008400098F49701A8016D2F7C2F8B2F9D2D01E02F
:100850000E94873520833183428353836483758369
:100860008683978381E0FCCE80E0FACE0895DB0199
:1008700014964D915C9115976D917C91DC01ED91F1
:10088000FC910280F381E02D0994AF92BF92CF9248
:10089000DF92EF92FF920F931F93CF93DF936C0140
:1008A0007B018B01040F151FEB015E01AE18BF0821
:1008B000C017D10759F06991D601ED91FC910190D3
:1008C000F081E02DC6010995892B79F7C501DF91EB
:1008D000CF911F910F91FF90EF90DF90CF90BF903D
:1008E000AF900895FC01538D448D252F30E0842F67
:1008F00090E0821B930B541710F0CF960895019748
:100900000895FC01918D828D981761F0A28DAE0F34
:10091000BF2FB11D5D968C91928D9F5F9F73928FBB
:1009200090E008958FEF9FEF0895FC01918D828DE7
:10093000981731F0828DE80FF11D858D90E00895B4
:100940008FEF9FEF0895FC01918D228D892F90E00C
:10095000805C9F4F821B91098F739927089585EEC4
:1009600095E00E94A30421E0892B09F420E0822F66
:10097000089580E090E0892B29F00E94AF04811156
:100980000C9400000895FC01A48DA80FB92FB11D8F
:10099000A35ABF4F2C91848D90E001968F739927B5
:1009A000848FA689B7892C93A089B1898C91837093
:1009B00080648C93938D848D981306C00288F3898C
:1009C000E02D80818F7D80830895EF92FF920F93B9
:1009D0001F93CF93DF93EC0181E0888F9B8D8C8DEB
:1009E00098131AC0E889F989808185FF15C09FB7DF
:1009F000F894EE89FF896083E889F98980818370A2
:100A0000806480839FBF81E090E0DF91CF911F9150
:100A10000F91FF90EF900895F62E0B8D10E00F5F71
:100A20001F4F0F731127E02E8C8D8E110CC00FB647
:100A300007FCFACFE889F989808185FFF5CFCE01DF
:100A40000E94C304F1CFEB8DEC0FFD2FF11DE35A93
:100A5000FF4FF0829FB7F8940B8FEA89FB89808162
:100A60008062CFCFCF93DF93EC01888D8823B9F0DC
:100A7000AA89BB89E889F9898C9185FD03C08081A9
:100A800086FD0DC00FB607FCF7CF8C9185FFF2CF26
:100A9000808185FFEDCFCE010E94C304E9CFDF91B5
:100AA000CF910895833081F028F4813099F082301D
:100AB000A9F008958730A9F08830C9F08430B1F4E6
:100AC000809180008F7D03C0809180008F7780931C
:100AD0008000089584B58F7784BD089584B58F7D97
:100AE000FBCF8091B0008F778093B0000895809104
:100AF000B0008F7DF9CFCF93DF93282F30E0F9013D
:100B0000E255FF4F8491F901E656FF4FD491F90168
:100B1000EA57FF4FC491CC23A1F081110E945205E6
:100B2000EC2FF0E0EE0FFF1FE458FF4FA591B491BA
:100B3000EC91ED2381E090E009F480E0DF91CF912A
:100B4000089580E090E0FACF1F93CF93DF93282F92
:100B500030E0F901E255FF4F8491F901E656FF4F6D
:100B6000D491F901EA57FF4FC491CC23A9F0162F75
:100B700081110E945205EC2FF0E0EE0FFF1FEE589E
:100B8000FF4FA591B4918FB7F894EC91111108C063
:100B9000D095DE23DC938FBFDF91CF911F91089515
:100BA000DE2BF8CF10927905109278051092C205CD
:100BB0001092E4051092C00581E08093BF05109269
:100BC0009A0561E082E10E94A40561E083E10E9450
:100BD000A405E9EBF0E080818E7F808380818D7FAA
:100BE000808388E48093B80085E48093BC0081EF23
:100BF00090E0909377058093760582EF90E0909354
:100C00007505809374050895CF93DF9390E0FC0100
:100C1000E656FF4F24918A579F4FFC018491882309
:100C2000C9F090E0880F991FFC01E859FF4FA5918A
:100C3000B491FC01EE58FF4FC591D49161110DC0E4
:100C40009FB7F8948C91209582238C9388812823D8
:100C500028839FBFDF91CF910895623051F49FB7F1
:100C6000F8943C91822F809583238C93E8812E2BDE
:100C7000EFCF8FB7F894EC912E2B2C938FBFEACF48
:100C80008E50806480937C0080917A008064809391
:100C90007A0080917A0086FDFCCF80917800909157
:100CA000790008953FB7F89480911205909113054B
:100CB000A0911405B091150526B5A89B05C02F3F3E
:100CC00019F00196A11DB11D3FBFBA2FA92F982F72
:100CD0008827BC01CD01620F711D811D911D42E06D
:100CE000660F771F881F991F4A95D1F708958F9235
:100CF0009F92AF92BF92CF92DF92EF92FF924B0101
:100D00005C010E9452066B017C010E9452066C1924
:100D10007D098E099F09683E734081059105A8F3FE
:100D200021E0821A9108A108B10888EEC80E83E07C
:100D3000D81EE11CF11C81149104A104B10429F70F
:100D4000FF90EF90DF90CF90BF90AF909F908F90EB
:100D500008952FB7F89460910E0570910F0580915A
:100D60001005909111052FBF089585ED8093BC006B
:100D70008091BC0084FDFCCF1092C00508952091A5
:100D8000EA04260F3327331F21323105ECF420917A
:100D9000C005FC0190E080E0243069F082E0089515
:100DA000A091EA042191AC0146535B4FA40FB52FEB
:100DB000B11D2C930196861798F38091EA04680F71
:100DC0006093EA0480E0089581E008950895E09139
:100DD000790580917805E81730F4F0E0E658FA4F8D
:100DE000808190E008958FEF9FEF089590917905AD
:100DF000809178052FEF3FEF981748F4E92FF0E046
:100E0000E658FA4F208130E09F5F90937905C90141
:100E10000895CF92DF92EF92FF920F931F93CF939B
:100E2000DF937C01CB018A012091C105222389F047
:100E3000EB016B01C40ED51ECC15DD0569F069917F
:100E4000D701ED91FC910190F081E02DC70109954A
:100E5000F3CF642F0E94BF06C801DF91CF911F918D
:100E60000F91FF90EF90DF90CF900895CF93DF9395
:100E70001F92CDB7DEB769832091C1052223F9F017
:100E80002091E405203258F021E030E0FC0133836A
:100E9000228390E080E00F90DF91CF9108958091C0
:100EA000C205E82FF0E0ED53FA4F998190838F5FF0
:100EB0008093C2058093E40581E090E0ECCF61E08F
:100EC000CE0101960E94BF06F7CFCF93C62F91E0C7
:100ED0009093C10590E69093E3051092C20510929D
:100EE000E405682F82E896E00E9436076C2F82E8BE
:100EF00096E00E94360781E0CF910C948D000F930D
:100F00001F93CF93DF938B0191E09093C10590E6FF
:100F10009093E3051092C2051092E405682F82E8D1
:100F200096E00E943607E801085F1F4F699182E84A
:100F300096E00E943607C017D107C1F781E0DF9124
:100F4000CF911F910F910C948D0090E080E0089557
:100F50008FE00E9440069093550580935405BC0194
:100F6000990F880B990B0E94543120E030E040EA41
:100F700050E40E94B33120E030E040E85AE30E94A0
:100F8000B33160932C0570932D0580932E059093BB
:100F90002F050895CF93DF9391E09093C10590E6DC
:100FA0009093E3051092C2051092E405682F82E841
:100FB00096E00E94360781E00E948D008091C00576
:100FC0008111FCCF81E08093C0051092BF059FEF97
:100FD0009093BE051092BD051092BC0580939B05B1
:100FE00080919B05806C80939B0580919A05813050
:100FF00061F510929A0580919B058093BB008091CA
:10100000BC0083FDF8CF85EC8093BC008091C005C7
:101010008130E1F38091BD05811119C08091BD053A
:10102000ECE9F5E0AAE7B5E0C0E0C81312C0109201
:101030007905C093780580917905C81771F082E829
:1010400096E00E94F606D82FF6CF85EEDDCF81E040
:10105000E7CF91919D93CF5FE8CF8D2FDF91CF9117
:101060000895CF93C0E1C80F8C2F0E94CA078C7FD0
:10107000682F62608C2FCF910C946507CF93DF931C
:10108000D82FC62F83E00E94CA0761E070E001C03C
:10109000660FDA95EAF7C13039F46095682383E08A
:1010A000DF91CF910C946507682BF9CF0F931F93B5
:1010B000CF938B01C0E1C80F8C2F0E94CA07682F05
:1010C000012B39F46F7D8C2FCF911F910F910C94D0
:1010D00065076062F8CFCF93DF93EC0160E08E810B
:1010E0000E94A40561E08E810E94A40560E08E81CB
:1010F0000E94A4058BE891E00197F1F7DF91CF9171
:101100000895CF92DF92EF92FF920F931F93CF93A8
:10111000DF936C017C0187E0E80EF11CD0E0C0E0B9
:10112000062F10E0B8010C2E02C0759567950A9441
:10113000E2F76170F70181917F010E94A405219679
:10114000C430D10579F7C601DF91CF911F910F917E
:10115000FF90EF90DF90CF900C946B08CF92DF92CE
:10116000EF92FF920F931F93CF93DF93EC01F62E34
:10117000642F8C810E94A4058D818F3F19F060E05F
:101180000E94A4050F2D10E08F8584FF25C06E01FD
:1011900087E0C80ED11CF12CE12CB8010E2C02C046
:1011A000759567950A94E2F76170F60181916F0178
:1011B0000E94A405FFEFEF1AFF0A88E0E816F10489
:1011C00061F7CE01DF91CF911F910F91FF90EF90CA
:1011D000DF90CF900C946B08B80184E0759567950B
:1011E0008A95E1F7CE010E9481086F2DCE01DF9133
:1011F000CF911F910F91FF90EF90DF90CF900C94C3
:10120000810840E0682F81E197E00C94AE08CF930D
:10121000DF93823029F49091200798609093200703
:10122000809324071092250780E48093260780E1AD
:101230008093270780E58093280761E08091150758
:101240000E940406809116078F3F19F061E00E940A
:10125000040661E0809117070E940406C1E1D7E00F
:101260009E01215137408091200784FD0BC084E00E
:1012700090E021962817390744F461E08E810E949E
:101280000406EECF88E090E0F4CF8BE39DE0019779
:10129000F1F760E0809115070E94A40560E080915D
:1012A00017070E94A405809116078F3F19F060E090
:1012B0000E94A4058091200784FD39C063E081E18C
:1012C00097E00E948108CBE4D6E4CE010197F1F7C4
:1012D00063E081E197E00E9481082197F1F763E0E4
:1012E00081E197E00E94810883E592E00197F1F7A0
:1012F00062E081E197E00E9481088091200780628E
:101300000E94010984E0809321078CE00E9401097A
:1013100081E00E9401098BE39FE10197F1F782E0F0
:101320008093220786E0DF91CF910C9401098062BF
:101330000E9401098BE496E40197F1F78091200760
:1013400080620E94010983E592E00197F1F78091A4
:10135000200780620E940109D0CF9091240769176D
:1013600010F06FEF690FE62FF0E0EF5EF84F948911
:10137000890F80680C94010941E00E94AE0881E069
:1013800090E008950F931F93CF93DF938B0128E094
:10139000829FC001112480640E940109E801085F56
:1013A0001F4F699181E197E00E94BC09C017D107E6
:1013B000C1F7DF91CF911F910F91089541E0682F00
:1013C00081E197E00E94AE0881E090E00895FC0181
:1013D00001900020E9F73197AF01481B590BBC0180
:1013E00081E197E00C9445048F929F92AF92BF9257
:1013F0000F931F93CF93DF93CDB7DEB7A1970FB6AF
:10140000F894DEBF0FBECDBF19A2423008F44AE007
:101410008E010F5D1F4F842E912CB12CA12CA501A4
:1014200094010E941434E62FB901CA01EA30F4F4A1
:10143000E05DD801EE938D01232B242B252B79F72A
:1014400090E080E0109719F0CD010E94E709A19685
:101450000FB6F894DEBF0FBECDBFDF91CF911F91C5
:101460000F91BF90AF909F908F900895E95CE1CF6E
:10147000CF92DF92EF92FF92CF93DF9397FF19C045
:101480006B017C018DE20E94DE09EC016627772763
:10149000CB016C197D098E099F094AE00E94F4096D
:1014A0008C0F9D1FDF91CF91FF90EF90DF90CF9039
:1014B00008954AE0DF91CF91FF90EF90DF90CF90B9
:1014C0000C94F409CF92DF92EF92FF92C090360510
:1014D000D0903705E0903805F09039058AE0C816BD
:1014E000D104E104F1041CF480E20E94DE0980E2F0
:1014F0000E94DE09C701B6010E94380A8EE20E94EE
:10150000DE0960913A0570913B0580913C05909110
:101510003D0520E432E44FE050E00E94363428EEEE
:1015200033E040E050E00E94363469017A01C09215
:101530003605D0923705E0923805F092390584E6F9
:10154000C816D104E104F10464F480E30E94DE09CA
:101550008AE0C816D104E104F1041CF480E30E947F
:10156000DE09C701B6010E94380A8EE20E94DE0938
:1015700060913A0570913B0580913C0590913D0545
:1015800028EE33E040E050E00E9436346B017C01ED
:10159000C0923605D0923705E0923805F0923905B1
:1015A00084E6C816D104E104F10464F480E30E94E7
:1015B000DE098AE0C816D104E104F1041CF480E3DA
:1015C0000E94DE09C701B601FF90EF90DF90CF9037
:1015D0000C94380A61E084E00E94AD096091AB018F
:1015E0007091AC018091AD019091AE0160933A058C
:1015F00070933B0580933C0590933D0520E432E4D5
:101600004FE050E00E943634209336053093370582
:1016100040933805509339050E94620A80E20C9489
:10162000DE090C94E7098091290590912A0561E073
:10163000019709F451C080E00E94AD0980916501D5
:1016400090916601A0916701B0916801843691057F
:10165000A105B10591F190F48A309105A105B1057C
:1016600031F182339105A105B10521F10197A10561
:10167000B105C1F58BE092E00C94110B883E23E09C
:101680009207A105B105F9F030F4843F9140A1051E
:10169000B105B1F00895803127E29207A105B105A7
:1016A000A9F0803A9648A140B10599F0089580E1EB
:1016B00092E0E2CF85E192E0DFCF8AE192E0DCCFF9
:1016C0008FE192E0D9CF84E292E0D6CF89E292E036
:1016D000D3CF8EE292E0D0CF80E00E94AD0983E3C9
:1016E00092E0CACF08954F925F926F927F928F924D
:1016F0009F92AF92BF92CF92DF92EF92FF920F93A1
:101700001F93CF936B017C01742EAC019B010E944F
:10171000EB33882399F088E392E0CF911F910F91EA
:10172000FF90EF90DF90CF90BF90AF909F908F9001
:101730007F906F905F904F900C94E709460157019E
:10174000E894B7F82FEF3FEF4FE75FE7C501B4012B
:101750000E94EB3381110DC02FEF3FEF4FE75FE7A2
:10176000C501B4010E944D3118161CF48CE392E0BF
:10177000D4CF2FEF3FEF4FE75FE4C701B6010E94E0
:10178000E63318161CF480E492E0C7CF2FEF3FEF4A
:101790004FE75FECC701B6010E944D3187FDF3CFE3
:1017A00020E030E0A901C701B6010E944D3110E0F0
:1017B00000E087FF08C08DE20E94DE098C01F7FA85
:1017C000F094F7F8F094C0E060E070E080E09FE310
:1017D0007C1641F020E030E040E251E40E944533C5
:1017E000CF5FF6CFA70196010E94D9322B013C01B1
:1017F0000E94B7334B015C014AE00E94F4097C016E
:10180000E00EF11ECC23B1F1C501B4010E945231AA
:101810009B01AC01C301B2010E94D8324B015C01B3
:101820008EE20E94DE09E80EF91EC15018F120E098
:1018300030E040E251E4C501B4010E94B3312B0114
:101840003C010E94B7334B01B12CA12C4AE0C501E9
:10185000B4010E94F409E80EF91EC501B4010E940A
:1018600052319B01AC01C301B2010E94D8324B013D
:101870005C01DBCFC701CF911F910F91FF90EF90DB
:10188000DF90CF90BF90AF909F908F907F906F90A0
:101890005F904F9008952F923F924F925F926F9278
:1018A0007F928F929F92AF92BF92CF92DF92EF92F0
:1018B000FF920F931F93CF93DF93CDB7DEB72D9792
:1018C0000FB6F894DEBF0FBECDBF3C01C982DA82ED
:1018D000EB82FC820D831E832F83388749875A87CA
:1018E0006B877C878AA18D873C2C2D2C9E2C502EBB
:1018F000412EB22EC984DA84EB84FC8484E190E02A
:101900000E94F5358C01FC01D082C182862D880FA2
:10191000880F880F845D0E94CA07F92DF3709F2EEF
:101920008C7F982AF8019282238234824CE0F694CC
:10193000E794D794C7944A95D1F7FC2DF07FCF2E2A
:101940008B2D8F70C82AF801C58246825782B80154
:1019500082E3F1E06F16710431F082E068167104E1
:1019600009F447C08AE20E947F0730E1F32EF60CAB
:101970008F2D0E94CA0791E0682FA9123CC06064B5
:101980008F2D0E946507E1E06E167104B1F1F2E05F
:101990006F167104B9F1A09204072CE2F22E8F2D7C
:1019A0000E94CA0783789D8591118C60E0E18E9E2C
:1019B000B0011124682B8F2D0E946507C8012D9658
:1019C0000FB6F894DEBF0FBECDBFDF91CF911F9150
:1019D0000F91FF90EF90DF90CF90BF90AF909F90CE
:1019E0008F907F906F905F904F903F902F900C94CE
:1019F00091368AE3B8CF6F7BC3CFA092050794E3FB
:101A0000F92ECDCFA09206078CE3F82EC8CF2F92E7
:101A10003F924F925F926F927F928F929F92AF927E
:101A2000BF92CF92DF92EF92FF920F931F93CF93CB
:101A3000DF93CDB7DEB76A970FB6F894DEBF0FBE5F
:101A4000CDBF2F8B3987488F598F6A877A8F1C01BA
:101A50001E8B0D8B60910D0770910E0780910F0703
:101A60009091100724E630E040E050E00E94BC3442
:101A7000522E632E742E852E962E788B8F87492EAC
:101A80008091070790910807A0910907B0910A0774
:101A90006C017D01FF0CCC08DC2C76019C01AD01B2
:101AA0006C2D7C2D8C2D9C2D0FE10E948735A12C57
:101AB000EAECBE2EFAE9CF2EABE3DA2EE12CF12CC4
:101AC00000E010E00E94E934A52CB62CC72CD82CDD
:101AD000E92CF8880F85142D0E9455340FE10E94DF
:101AE000A23529833A834B835C836D837E838F8306
:101AF000988789819A81AB81BC81BB0F880B982F15
:101B0000DC018B879C87AD87BE87252D362D472D21
:101B1000582D692D7F2D8F85942DA980BA80CB807B
:101B2000DC80EB84FE2C0E2D1E2D0E94BD352983FA
:101B30003B874F87588B698B7A8B8B8B9C8B8F88DD
:101B40009A8C282D3985488D598D6A85792DC1014A
:101B5000211534404B46544F644171058105910570
:101B600069F060F0812CB4E0B987EBE6E88FF4EF20
:101B7000F98F84E18A87912C212C312C282D3985ED
:101B8000488D598D6A85792DC10121153845474405
:101B9000584F6D4071058105910560F4812CB8E5C1
:101BA000B987E7E4E88FF8EFF98F8DE08A87912C09
:101BB000212C312CA980BB84CF84D888E988FA886D
:101BC0000B891C89282D3985488D598D6A85792D79
:101BD000C1010E941A3529013A011FE0A12E9FE0A0
:101BE000491651046104710440F0ABE54A165104F2
:101BF00061047104D0F0BAE5AB2EB12CC12CD12C0C
:101C0000E12CF12C00E010E029813B854F855889BB
:101C100069897A898B899C890E945534822E3987FB
:101C2000488F598F6A87972E1C01A980BB84CF8467
:101C3000D888E988FA880B891C89282D3985488D30
:101C4000598D6A85792DC1010E941835AA24AA945C
:101C5000BB24BA94AFE0CA2ED12CE12CF12C00E0C9
:101C600010E00E945534A980BB84CF84D888E988CD
:101C7000FA880B891C890E941A35C901DA01812C66
:101C8000912C540183940097A105B10531F088246B
:101C90008A94982CEFE0AE2EB12CBC01CD0127E048
:101CA000660F771F881F991F2A95D1F7A501940108
:101CB0000E941434362E272E182F67E0440C551C32
:101CC000661C771C6A95D1F7B2E05B1A610871084F
:101CD000420E531E641E751E84E190E00E94F5358D
:101CE0009A838983FC0190828182862D837082830E
:101CF000538244827CE0B694A794979487947A9513
:101D0000D1F7F82DF07F8F2E812AA981BA811596FF
:101D10008C92159716962C92169717963C921797B9
:101D2000ED89FE89BD018AE1EF2B19F069817A8185
:101D300082E20E947F0789819A816A960FB6F894A1
:101D4000DEBF0FBECDBFDF91CF911F910F91FF90EE
:101D5000EF90DF90CF90BF90AF909F908F907F904B
:101D60006F905F904F903F902F900C9491362F92F0
:101D70003F924F925F926F927F928F929F92AF921B
:101D8000BF92CF92DF92EF92FF920F931F93CF9368
:101D9000DF93CDB7DEB7AA970FB6F894DEBF0FBEBC
:101DA000CDBF622E298F732E3A8F4B8F5C8F6D8F34
:101DB0007E8F8F8F98A319A708A793012F3F3443D5
:101DC0004C405105610571058105910509F050F4FC
:101DD000198E85E38A8F8CE08B8F1C8E1D8E1E8E54
:101DE0001F8E18A2298D3A8D4B8D5C8D6D8D7E8D49
:101DF0008F8D98A12115304A4C4A594B634071058B
:101E00008105910569F060F0198E80EA8A8F8CEA6D
:101E10008B8F89EB8C8F83E08D8F1E8E1F8E18A287
:101E2000CE0149960E94F7028FA3798CBA8DAB8DB3
:101E3000FC8DED8D6E8C5F8C48A0272D3B2F4A2F9B
:101E40005F2F6E2F762D852D942D2F3F05ED3007BA
:101E500001E140070EE7500703E0600771058105C7
:101E6000910511F008F09EC0CE010D964C01A12CF9
:101E7000EEE2BE2EF9E5CF2EA6E7DA2EB1E1EB2E8B
:101E8000F12C00E010E0852D942D0E94F300798D57
:101E90006A8D5B8D4C8D3D8D2E8D9F8D88A1E8A523
:101EA000F9A5E130F10509F445C0329709F45EC0A7
:101EB0007093EC066093ED065093EE064093EF06A8
:101EC0003093F0062093F1069093F2068093F30688
:101ED00080E019A2412CFEE2FAA309E50BA316E764
:101EE0001CA391E19DA3512C612C712C8F938FA089
:101EF000A82ECD84DE84EF84F88809891A892B897D
:101F00003C894D895E896F89788D88A599A50E9445
:101F10004B0C0F9099A1913009F0FBC08101242D49
:101F20003AA14BA15CA16DA1752DC3010E94070DC3
:101F300019A2EFC07093F4066093F5065093F6066D
:101F40004093F7063093F8062093F9069093FA062B
:101F50008093FB0680E019A2412CEEE2EAA3F9E5AA
:101F6000FBA306E70CA311E11DA3BDCF7093FC06F4
:101F70006093FD065093FE064093FF0630930007E2
:101F800020930107909302078093030780E019A232
:101F9000412C9EE29AA3E9E5EBA3F6E7FCA301E15D
:101FA0000DA3A1CFCE010D964C01A12CB12CC12CBB
:101FB000D12CE12CF12C00E010E0852D942D0E9415
:101FC000F300298C3A8CBB8DAC8DFD8DEE8D08A570
:101FD00019A50130110509F44EC00230110509F4AC
:101FE000A5C100E010E091014B2F5A2F6F2F7E2FDB
:101FF0008F8D98A10E94F300422E3AA34BA35CA3BD
:102000006DA3572E3C0170E060E090E080E00E94FC
:1020100056084092DC069AA19093DD06EBA1E0936E
:10202000DE06FCA1F093DF060DA10093E0065092BE
:10203000E1066092E2067092E306898D8093EC06D9
:102040008A8D8093ED068B8D8093EE068C8D809328
:10205000EF068D8D8093F0068E8D8093F1068F8D27
:102060008093F20688A18093F30681E011E019A322
:10207000312C212C3BCF0F8D09A318A11EA3109149
:102080000C07123009F019C191014B2F5A2F6F2FF5
:102090007E2F802F9EA130584A4156406109710918
:1020A000810991092F37304E4247584962407105E6
:1020B0008105910509F008F446C02091FC06309195
:1020C000FD064091FE065091FF0660910007709159
:1020D000010780910207909103075101CB2EDA2E60
:1020E000EF2EFE2E09A11EA10E94C63561F11092AD
:1020F000F4061092F5061092F6061092F70610926A
:10210000F8061092F9061092FA061092FB0611E0FA
:1021100019A389A1AA960FB6F894DEBF0FBECDBF52
:10212000DF91CF911F910F91FF90EF90DF90CF90B3
:10213000BF90AF909F908F907F906F905F904F90E7
:102140003F902F9008954090E4068091E5068AA381
:102150009091E6069BA30091E7060CA31091E80678
:102160001DA35090E9066090EA067090EB06CE0140
:102170000D964C01A42CBAA0CBA0D02EE12EF52CAC
:10218000830191014B2F5A2F6F2F7E2F89A19EA182
:102190000E94F30061E070E081E090E00E94560848
:1021A00019A2298D3A8D4B8D5C8D6D8D7E8D8F8D15
:1021B00098A130584A415640610971098109910935
:1021C0002F37304E424758496240710581059105CD
:1021D00009F008F4A7C081E080930C072091FC0669
:1021E0003091FD064091FE065091FF066091000778
:1021F000709101078091020790910307A0E00E946F
:10220000CF35F1F18CEF96E00E94F7028FA3A090FA
:10221000E406B090E506C090E606D090E706E090B0
:10222000E806F090E9060091EA061091EB0620918D
:10223000FC063091FD064091FE065091FF0660912C
:10224000000770910107CE0101964C0180910207B1
:10225000909103070E94F3001F928FA0A12CC980C8
:10226000DA80EB80FC800D811E812F8138854985C5
:102270005A856B857C8582E090E00E944B0C0F9024
:10228000898D8093F4068A8D8093F5068B8D8093DB
:10229000F6068C8D8093F7068D8D8093F8068E8DD3
:1022A0008093F9068F8D8093FA0688A18093FB06B0
:1022B00081E022242394312C19CE2093E40630931C
:1022C000E5064093E6065093E7066093E8067093B0
:1022D000E9068093EA069093EB068E01035F1F4F99
:1022E0004801A12CB12CC12CD12CE12CF12C00E007
:1022F00010E091014B2F5A2F6F2F7E2F89A19EA1A5
:102300000E94F300422E3AA34BA35CA36DA3572E69
:102310003C0161E070E081E090E00E94560811E02D
:1023200019A33FCF88E080930C07AACF00910C0738
:1023300009A31F8D1EA308A10AA719A1113009F036
:10234000F9C091014B2F5A2F6F2F7E2F8EA1902F06
:1023500030584A41564061097109810991092F3766
:10236000304E42475849624071058105910561F13F
:1023700058F12091FC063091FD064091FE065091E7
:10238000FF0660910007709101078091020790910C
:1023900003075101CB2EDA2EEF2EFE2E0EA11AA529
:1023A0000E94C63589F01092FC061092FD0610922C
:1023B000FE061092FF06109200071092010710927D
:1023C000020710920307A5CE4090E4061091E5069F
:1023D0001AA38091E6068BA39091E7069CA3009137
:1023E000E8060DA35090E9066090EA067090EB06AF
:1023F000CE010D964C01A42CB12ECBA0DCA0E02E7A
:10240000F52C830191014B2F5A2F6F2F7E2F8EA118
:102410009AA50E94F30061E070E082E090E00E94E3
:10242000560819A2298D3A8D4B8D5C8D6D8D7E8D50
:102430008F8D98A130584A41564061097109810930
:1024400091092F37304E4247584962407105810546
:10245000910509F008F4A3C082E080930C07209155
:10246000F4063091F5064091F6065091F70660911A
:10247000F8067091F9068091FA069091FB06A0E0AB
:102480000E94CF35F1F184EF96E00E94F7028FA30E
:10249000A090E406B090E506C090E606D090E7066E
:1024A000E090E806F090E9060091EA061091EB064C
:1024B0002091F4063091F5064091F6065091F7060A
:1024C0006091F8067091F906CE0101964C01809159
:1024D000FA069091FB060E94F3001F928FA0A12C98
:1024E000C980DA80EB80FC800D811E812F813885C8
:1024F00049855A856B857C8581E090E00E944B0C74
:102500000F90898D8093FC068A8D8093FD068B8DBC
:102510008093FE068C8D8093FF068D8D809300073F
:102520008E8D809301078F8D8093020788A1809301
:102530000307BECE2093E4063093E5064093E606FB
:102540005093E7066093E8067093E9068093EA06E5
:102550009093EB068E01035F1F4F4801A12CB12C15
:10256000C12CD12CE12CF12C00E010E091014B2F7B
:102570005A2F6F2F7E2F8EA19AA50E94F300422E14
:102580003AA34BA35CA36DA3572E3C0161E070E01E
:1025900082E090E00E94560811E019A343CF88E042
:1025A00080930C07AECFCF93DF93EC0188819981A4
:1025B000009711F00E949136198218821D821C82A8
:1025C0001B821A82DF91CF910895FC018081918155
:1025D0000C9491360F931F93CF93DF938C01EB01F3
:1025E0000E9471328883C80101960E9471328983EA
:1025F000CE01DF91CF911F910F910895CF92DF927D
:10260000EF92FF920F931F93CF93DF93EB017B0128
:1026100024E0E20EF11C8B016C01C61AD70AC60138
:10262000800F911F0E947132F80181938F01EE1586
:10263000FF05A9F7CE01DF91CF911F910F91FF9078
:10264000EF90DF90CF900895CF93DF93C091230553
:10265000D091240568E271E08AEA90E0209739F091
:10266000C130D105E1F564E271E08FEA90E00E94AB
:10267000FE12FC0180819181A281B3818093B5011A
:102680009093B601A093B701B093B801109246059C
:1026900010924705109248051092490564E171E0D7
:1026A00083EC90E0C530D105C1F50E94FE12FC011B
:1026B00080819181A281B3818093B5019093B6010D
:1026C000A093B701B093B801109246051092470548
:1026D0001092480510924905DF91CF910895C230BC
:1026E000D10519F560E271E084EB90E00E94FE12E2
:1026F000FC0180819181A281B3818093B501909387
:10270000B601A093B701B093B8011092460510929C
:102710004705109248051092490560E171E088EC88
:1027200090E0C630D10509F21EC0C330D10561F575
:102730006CE171E089EB90E00E94FE12FC01808167
:102740009181A281B3818093B5019093B601A0934A
:10275000B701B093B8011092460510924705109248
:102760004805109249056CE071E08DEC90E0C730AF
:10277000D10509F49ACF68E071E082ED90E0C830AD
:10278000D10509F492CF1FC0C430D10509F086CF1E
:1027900068E171E08EEB90E00E94FE12FC01808106
:1027A0009181A281B3818093B5019093B601A093EA
:1027B000B701B093B80110924605109247051092E8
:1027C000480510924905299709F086CF60E071E02D
:1027D00087ED90E06ACFCF93DF93EB010E947132D7
:1027E0008883CE01DF91CF9108950F931F93CF93EC
:1027F000DF93EC0188819981009759F02A813B8110
:102800002617370730F081E0DF91CF911F910F91AC
:1028100008958B016F5F7F4F0E941A37009759F020
:10282000998388831B830A832C813D81232B59F74D
:10283000FC011082E8CF80E0E7CFEF92FF920F9388
:102840001F93CF93DF936115710541F480E0DF9111
:10285000CF911F910F91FF90EF9008954115510571
:10286000B1F07B01EC010C811D81040F151FB80133
:102870000E94F513882351F3288139818C819D8131
:10288000B701820F931F0E94E9371D830C8381E0FB
:10289000DECFFC0101900020E9F73197AF01481B22
:1028A000590BBC018CEA96E00C941D14EF92FF9238
:1028B0000F931F93CF93DF93EC017B018A01BA0141
:1028C0000E94F51381110BC0CE010E94D312CE01DC
:1028D000DF91CF911F910F91FF90EF9008951D838D
:1028E0000C83B701888199810E94E937F0CFFB0101
:1028F00001900020E9F73197AF01461B570B0C946C
:102900005614FC01118210821382128215821482E5
:10291000FB0101900020E9F73197AF01461B570BEF
:102920000C945614FF920F931F93CF93DF93EC01F7
:10293000F62E08811981C8010E947132F81621F023
:102940006F2DC8010E947932CE01DF91CF911F9186
:102950000F91FF900895EF92FF920F931F93CF93E3
:10296000DF9300D0CDB7DEB705EB11E0855B91407A
:102970007C01C701800F911F9A838983F8016191BF
:102980008F01CE0101960E949214F1E0093B1F07CE
:1029900081F785EB91E00F900F90DF91CF911F9120
:1029A0000F91FF90EF9008958091B5019091B6013D
:1029B000A091B701B091B8018032914AA740B1050A
:1029C000C8F08091B5019091B601A091B701B09186
:1029D000B8018038994BAA42B10560F42A982B9827
:1029E0002C982D9810922405109223058AEA90E0E5
:1029F0000C94AB148091B5019091B601A091B701F0
:102A0000B091B8018038994BAA42B10570F080911D
:102A1000B5019091B601A091B701B091B801803491
:102A20009B44AC44B10508F463C08091B50190911A
:102A3000B601A091B701B091B80180349B44AC4479
:102A4000B10508F062C08091B5019091B601A091E6
:102A5000B701B091B80181159241AA47B10508F0BC
:102A60006FC08091B5019091B601A091B701B0916E
:102A7000B80181159B41A74BB10508F07CC080913E
:102A8000B5019091B601A091B701B091B80181153F
:102A90009442A44FB10508F089C08091B50190918E
:102AA000B601A091B701B091B801803C9A4EA14205
:102AB000B14008F096C08091B5019091B601A09107
:102AC000B701B091B8018038914BAF44B14008F0E4
:102AD000A3C08091B5019091B601A091B701B091CA
:102AE000B801803C9C4FAB49B14008F0B0C008959C
:102AF0002A9A2B982C982D9881E090E090932405A9
:102B0000809323058FEA90E073CF8091B501909177
:102B1000B601A091B701B091B80181159241AA47C1
:102B2000B10508F090CF2A982B9A2C982D9882E026
:102B300090E0909324058093230584EB90E058CF98
:102B40008091B5019091B601A091B701B091B80103
:102B500081159B41A74BB10508F083CF2A9A2B9A88
:102B60002C982D9883E090E0909324058093230582
:102B700089EB90E03DCF8091B5019091B601A09195
:102B8000B701B091B80181159442A44FB10508F086
:102B900076CF2A982B982C9A2D9884E090E09093E9
:102BA0002405809323058EEB90E022CF8091B50120
:102BB0009091B601A091B701B091B801803C9A4EB6
:102BC000A142B14008F069CF2A9A2B982C9A2D98EF
:102BD00085E090E0909324058093230583EC90E0BA
:102BE00007CF8091B5019091B601A091B701B09146
:102BF000B8018038914BAF44B14008F05CCF2A98BF
:102C00002B9A2C9A2D9886E090E09093240580933F
:102C1000230588EC90E0ECCE8091B5019091B6014F
:102C2000A091B701B091B801803C9C4FAB49B14035
:102C300008F04FCF2A9A2B9A2C9A2D9887E090E093
:102C400090932405809323058DEC90E0D1CE809164
:102C5000B5019091B601A091B701B091B80181384A
:102C6000934CA94CB14068F42A982B982C982D9A33
:102C700088E090E0909324058093230582ED90E016
:102C8000B7CE0895AF92BF92CF92DF92EF92FF92AC
:102C90000F931F93CF93DF9300D0CDB7DEB78B0197
:102CA0006B0124E0C20ED11C7B015C01A61AB70A9D
:102CB000C5018E0D9F1D9A838983F70161917F0164
:102CC000CE0101960E949214EC14FD0489F7C8010C
:102CD0000F900F90DF91CF911F910F91FF90EF9088
:102CE000DF90CF90BF90AF900895EF92FF920F9337
:102CF0001F93CF93DF9300D0CDB7DEB78C017B015C
:102D00009A838983FB016081CE0101960E9492140F
:102D10000F5F1F4F1A830983F7016181CE0101966E
:102D20000E949214C7010F900F90DF91CF911F91D5
:102D30000F91FF90EF9008950F931F93CF93DF9320
:102D400000D0CDB7DEB78B019A838983FB01608108
:102D5000CE0101960E949214C8010F900F90DF914E
:102D6000CF911F910F9108958F929F92AF92BF9232
:102D7000FF920F931F93CF93DF93EC01F0907005B8
:102D80000091720510917305F11052C002301105C7
:102D900009F44EC08130910509F0B6C080912B0531
:102DA0008F5F873008F0AEC080932B05409165019E
:102DB0005091660160916701709168018091B50141
:102DC0009091B601A091B701B091B801840F951F01
:102DD000A61FB71F8093B5019093B601A093B701CA
:102DE000B093B8016091B5017091B6018091B701BF
:102DF0009091B80120916501309166014091670181
:102E0000509168018090650190906601A0906701E3
:102E1000B09068010E941434C501B4010E94F033DF
:102E20006093B5017093B6018093B7019093B80198
:102E30008091B5019091B601A091B701B091B80110
:102E40008130914EA54FB54060F080E091EEA5EF46
:102E5000B5E08093B5019093B601A093B701B0930C
:102E6000B8018091B5019091B601A091B701B091E0
:102E7000B8018032914AA740B10560F480E291EA3E
:102E8000A7E0B0E08093B5019093B601A093B7019D
:102E9000B093B80121E0F212BBC0C130D10509F0F6
:102EA00082C0409165015091660160916701709107
:102EB00068018091460590914705A0914805B09121
:102EC0004905840F951FA61FB71F80934605909351
:102ED0004705A0934805B09349050130110509F055
:102EE000D0C08091600590916105A0916205B0917C
:102EF00063058093B5019093B601A093B701B09399
:102F0000B8019DC087E050CF019609F091CF409164
:102F1000650150916601609167017091680180912F
:102F2000B5019091B601A091B701B091B801841B91
:102F3000950BA60BB70B8093B5019093B601A093A8
:102F4000B701B093B8016091B5017091B60180915D
:102F5000B7019091B80120916501309166014091CF
:102F60006701509168018090650190906601A09082
:102F70006701B09068010E941434C501B4010E9439
:102F8000F0336093B5017093B6018093B7019093CD
:102F9000B80180912B058150823018F080932B0569
:102FA00047CF81E0FBCFCF3FDC0709F04CC3409116
:102FB000650150916601609167017091680180918F
:102FC000460590914705A0914805B0914905841B9D
:102FD000950BA60BB70B8093460590934705A093DE
:102FE0004805B09349050130110509F04AC08091A8
:102FF000600590916105A0916205B0916305809391
:10300000B5019093B601A093B701B093B801FAC18E
:1030100001301105B1F58091600590916105A09195
:103020006205B09163058093B5019093B601A093BA
:10303000B701B093B801C130D10509F0DFC14091AB
:1030400065015091660160916701709168018091FE
:10305000730190917401A0917501B0917601840F74
:10306000951FA61FB71F8093730190937401A093BF
:103070007501B093760163E771E08AE190E00E9408
:1030800042168091720590917305029709F041C034
:103090008091600590916105A0916205B0916305F2
:1030A0008093B5019093B601A093B701B093B80196
:1030B0006AE175E08FE090E00E94FE12FC018081E1
:1030C0009181A281B3818093B0019093B101A093CB
:1030D000B201B093B301C130D10509F0A8C140914C
:1030E0006501509166016091670170916801840FDC
:1030F000951FA61FB71F8093B0019093B101A093B5
:10310000B201B093B30160EB71E08FE090E00E94F8
:10311000421680917205909173050397B1F58091E5
:10312000600590916105A0916205B091630580935F
:10313000B5019093B601A093B701B093B801C13027
:10314000D10509F095C140916501509166016091EA
:103150006701709168018091AB019091AC01A091E1
:10316000AD01B091AE01840F951FA61FB71F8093CC
:10317000AB019093AC01A093AD01B093AE016BEAAB
:1031800071E085E190E00E94421680917205909175
:103190007305049719F58091600590916105A091E0
:1031A0006205B09163058093B5019093B601A09339
:1031B000B701B093B801C130D10509F090C168E4FE
:1031C00072E084E996E00E94771481E08093AF0179
:1031D0006FEA71E08DE090E00E949C16809172058C
:1031E00090917305059719F580916005909161059F
:1031F000A0916205B09163058093B5019093B601EB
:10320000A093B701B093B801C130D10509F074C1E2
:1032100068E472E08AE996E00E94771481E0809386
:10322000B40164EB71E090E080E00E949C16809114
:103230007205909173050697B9F58091600590919C
:103240006105A0916205B09163058093B5019093EB
:10325000B601A093B701B093B801C130D10509F010
:103260005DC180916F0190917001A0917101B09149
:103270007201805F984DAF4FBF4F8038F3EC9F07CE
:10328000F9ECAF07F1E0BF070CF043C180936F0189
:1032900090937001A0937101B09372016FE671E099
:1032A00088E290E00E944216809172059091730529
:1032B0000797B1F58091600590916105A091620535
:1032C000B09163058093B5019093B601A093B701C7
:1032D000B093B801C130D10509F046C140916501F4
:1032E000509166016091670170916801809130058D
:1032F00090913105A0913205B0913305840F951F4F
:10330000A61FB71F8093300590933105A093320517
:10331000B093330560E375E084E290E00E944216CA
:1033200080917205909173050897C9F5C130D10558
:1033300009F033C18091600590916105A09162050B
:10334000B09163058093B5019093B601A093B70146
:10335000B093B8016FE971E088E290E00E94FE123C
:10336000409165015091660160916701709168011B
:10337000FC0180819181A281B381840F951FA61FDA
:10338000B71F80939F019093A001A093A101B093D8
:10339000A2016FE971E088E290E00E9442168091FC
:1033A0007205909173058930910509F030C18091C3
:1033B000600590916105A0916205B09163058093CD
:1033C000B5019093B601A093B701B093B80164E43E
:1033D00072E0CF3FDC0729F0219709F02AC168E4A9
:1033E00072E08EE896E0DF91CF911F910F91FF90F0
:1033F000BF90AF909F908F900C947714CF3FDC07D5
:1034000009F039CE409165015091660160916701E4
:10341000709168018091730190917401A091750180
:10342000B0917601841B950BA60BB70B1CCECF3F3A
:10343000DC0709F068CEB7FD66CE4091650150917A
:1034400066016091670170916801841B950BA60B62
:10345000B70B181619061A061B060CF44CCE109260
:10346000B0011092B1011092B2011092B3014BCE93
:10347000CF3FDC0709F083CE8091AB019091AC0186
:10348000A091AD01B091AE01B7FD79CE409165013B
:10349000509166016091670170916801841B950BE2
:1034A000A60BB70B181619061A061B060CF45FCEEE
:1034B0001092AB011092AC011092AD011092AE01CE
:1034C00064E472E084E996E00E9477141092AF0100
:1034D0006FEA71E08DE090E00E949C1650CECF3FE5
:1034E000DC0709F075CE64E472E084E996E00E949E
:1034F00077141092AF016CCECF3FDC0709F091CE6C
:1035000064E472E08AE996E00E9477141092B401B4
:1035100088CE80E893ECA9ECB1E0B8CECF3FDC07D1
:1035200009F0BCCE8093B5019093B601A093B7018A
:10353000B093B80180916F0190917001A0917101D9
:10354000B091720180519742A109B1098130E6E33F
:103550009E07EEE6AE07E1E0BE070CF097CE80E0F6
:1035600096E3AEE6B1E092CECF3FDC0709F0D2CED3
:103570004091650150916601609167017091680109
:103580008091300590913105A0913205B0913305BD
:10359000841B950BA60BB70BB5CECF3FDC0709F00C
:1035A000FECE8091600590916105A0916205B09179
:1035B00063058093B5019093B601A093B701B093D2
:1035C000B8016FE971E088E290E00E94FE1240913C
:1035D0006501509166016091670170916801FC017D
:1035E00080819181A281B381841B950BA60BB70BBF
:1035F000181619061A061B060CF4C3CE10929F016A
:103600001092A0011092A1011092A201C2CE0A97BD
:1036100081F48091600590916105A0916205B0915F
:1036200063058093B5019093B601A093B701B09361
:10363000B801DF91CF911F910F91FF90BF90AF9094
:103640009F908F9008950130110509F01ACD809157
:10365000600590916105A0916205B091630580932A
:10366000B5019093B601A093B701B093B80103CD13
:103670001F920F920FB60F9211242F933F934F93E7
:103680005F936F937F938F939F93AF93BF93EF93CA
:10369000FF9385EE95E00E94C304FF91EF91BF91E7
:1036A000AF919F918F917F916F915F914F913F91DA
:1036B0002F910F900FBE0F901F9018951F920F9291
:1036C0000FB60F9211242F938F939F93EF93FF9335
:1036D000E091F505F091F6058081E091FB05F09110
:1036E000FC0582FD1BC090818091FE058F5F8F736A
:1036F0002091FF05821741F0E091FE05F0E0EB51CB
:10370000FA4F958F8093FE05FF91EF919F918F91D6
:103710002F910F900FBE0F901F9018958081F4CFBE
:103720001F920F920FB60F9211242F933F938F93F6
:103730009F93AF93BF9380910E0590910F05A09139
:103740001005B091110530910D0523E0230F2D37A1
:1037500058F50196A11DB11D20930D0580930E050E
:1037600090930F05A0931005B09311058091120559
:1037700090911305A0911405B09115050196A11D16
:10378000B11D8093120590931305A0931405B09377
:103790001505BF91AF919F918F913F912F910F9000
:1037A0000FBE0F901F90189526E8230F0296A11DBB
:1037B000B11DD2CF1F920F920FB60F9211242F93EB
:1037C0003F934F935F936F937F938F939F93AF93A9
:1037D000BF93EF93FF938091B900887F803609F4FF
:1037E0004AC0F0F5883209F4A7C018F5803109F411
:1037F0009BC0B8F4882309F4F9C0883009F494C058
:10380000FF91EF91BF91AF919F918F917F916F91B8
:103810005F914F913F912F910F900FBE0F901F908E
:103820001895883109F488C0803251F78093BE051D
:1038300014C0803409F49DC040F48033B9F3883358
:10384000F9F68093BE0585ECB0C0803509F485C0DB
:10385000883509F496C0883499F60E94B506D0CF11
:10386000883909F48CC038F5883729F050F4883647
:1038700011F0803729F683E08093C00510920C0583
:1038800057C0883809F47BC0803919F0803809F0B6
:10389000B7CF80910C05803208F071C0E0910C0523
:1038A00081E08E0F80930C058091BB00F0E0E45125
:1038B000FB4F80833DC0803B39F0E0F4803A09F44F
:1038C00079C0883A09F09CCF84E08093C0051092BB
:1038D000EB041092EA04E0917605F09177050995E2
:1038E0008091EA0481110FC081E08093EA04109274
:1038F000CA0409C0803C09F4A6CF883C09F4A3CFD0
:10390000883B09F07DCFE091EB0481E08E0F80933E
:10391000EB04F0E0E653FB4F80818093BB00909175
:10392000EB048091EA0429C080919B058093BB0041
:1039300085EC8093BC0064CF9091BD058091BC055F
:10394000981758F5E091BD0581E08E0F8093BD0575
:10395000F0E0E456FA4F8081E9CFE091BD0581E0C7
:103960008E0F8093BD058091BB00F0E0E456FA4FC6
:1039700080839091BD058091BC059817C8F285E8B9
:10398000D8CFE091BD0581E08E0F8093BD05809179
:10399000BB00F0E0E456FA4F80838091BF058111AF
:1039A0005CCF81E080939A0584EA8093BC001092FA
:1039B000C00526CF85EC8093BC001092C005809195
:1039C0000C05803230F4E0910C05F0E0E451FB4F3F
:1039D000108260910C0570E0E0917405F09175051E
:1039E0008CEE94E0099510920C050ACF1092BE055A
:1039F00034CF1F920F920FB60F921124CF92DF9205
:103A0000EF92FF920F931F932F933F934F935F93E8
:103A10006F937F938F939F93AF93BF93CF93DF93D6
:103A2000EF93FF938091D2060E947B05EC01809179
:103A3000D1060E947B059091D0069F70CC0FDD1FB0
:103A4000C82B24E0929FC001112481549E4FC80FBF
:103A5000D92FD11DC881C093D006C07361F10E94D7
:103A6000A9060091160510911705209118053091AF
:103A700019056B017C01C01AD10AE20AF30A970109
:103A8000860100931F051093200520932105309394
:103A9000220560931605709317058093180590937F
:103AA000190581E090E0C03121F0C03221F48FEFA0
:103AB0009FEF0E94B416FF91EF91DF91CF91BF91DC
:103AC000AF919F918F917F916F915F914F913F91B6
:103AD0002F911F910F91FF90EF90DF90CF900F905B
:103AE0000FBE0F901F901895CF93DF93E5EEF5E092
:103AF0001382128288EE93E0A0E0B0E08483958385
:103B0000A683B7832FED31E03183208325EC30E0AD
:103B10003587248724EC30E03787268720EC30E097
:103B2000318B208B21EC30E0338B228B22EC30E088
:103B3000358B248B26EC30E0378B268B118E128E42
:103B4000138E148EE2E8F6E013821282848395834A
:103B5000A683B78381EF91E091838083E1E1F7E071
:103B60001382128283E092E09183808389E08483D0
:103B70008FEF8583C8E0C68387E0878386E08087F0
:103B800085E0818784E082871386148615861686F1
:103B9000178681E00E940709E3EDF6E0C0AFC1AFF0
:103BA00011AA12AA13AA11861286138614861586E4
:103BB00016861786108A118A128A138A148A158A21
:103BC000168A178A108E118E128E138E148E158EF1
:103BD000168E178E10A211A212A213A214A215A261
:103BE00016A217A210A611A612A613A614A615A611
:103BF00016A617A610AA80E498E7ADE7B1E082AF59
:103C000093AFA4AFB5AFC0EDD6E083E0898382E087
:103C10008A8360E083E00E94040660E08A810E945B
:103C2000040661E089810E94A40561E08A810E9406
:103C3000A40518826CE472E08AEC96E00E9481147C
:103C40006EE472E084EC96E00E94811462E572E01A
:103C50008EEB96E00E94811469E474E088EB96E0B4
:103C60000E94811469E474E082EB96E00E94811462
:103C700069E474E08CEA96E00E94811469E474E0DF
:103C800086EA96E00E94811469E474E080EA96E096
:103C90000E94811468E472E08AE996E00E9481142F
:103CA00068E472E084E996E00E94811464E472E0C2
:103CB0008EE896E0DF91CF910C948114CF93DF933F
:103CC000CDB7DEB7A7970FB6F894DEBF0FBECDBF56
:103CD000789484B5826084BD84B5816084BD85B5E7
:103CE000826085BD85B5816085BD80916E008160F3
:103CF00080936E0010928100809181008260809399
:103D0000810080918100816080938100809180009A
:103D10008160809380008091B10084608093B100C5
:103D20008091B00081608093B00080917A008460BF
:103D300080937A0080917A00826080937A008091EB
:103D40007A00816080937A0080917A008068809305
:103D50007A001092C100E091F505F091F60582E03D
:103D60008083E091F105F091F2051082E091F30576
:103D7000F091F4058FEC80831092FD05E091F90538
:103D8000F091FA0586E08083E091F705F091F8055F
:103D9000808180618083E091F705F091F805808152
:103DA00088608083E091F705F091F8058081806854
:103DB0008083E091F705F091F80580818F7D808305
:103DC00082E00E94070981E00E9401098BE39FE1E4
:103DD0000197F1F70E94D20561E08AE00E94040693
:103DE00061E08BE00E94040661E08CE00E94040622
:103DF00061E08DE00E94040660E08FE00E9404060E
:103E000061E080E10E94040661E081E10E94040615
:103E10006CE571E081E00E94C20964E571E082E036
:103E20000E94C2096CE471E083E00E94C20964E46C
:103E300071E084E00E94C2096CE371E085E00E94B9
:103E4000C20964E371E086E00E94C2096CE271E09D
:103E500087E00E94C2096EE175E089E090E00E946F
:103E6000EB13DC018C91833911F40C94782964EB09
:103E700071E090E080E00E949C1683E990E09A83D4
:103E80008983BE016F5F7F4F89E090E00E947516C5
:103E90006FEA71E08DE090E00E949C1660EB71E0AB
:103EA0008FE090E00E9442166BEA71E085E190E0BD
:103EB0000E94421663E771E08AE190E00E94421698
:103EC0008FE190E00E94AB1463EA71E084E290E03D
:103ED0000E9442166FE671E088E290E00E9442166E
:103EE00069E671E087E390E00E94751666E475E08C
:103EF0008CE390E00E9442166FE971E08AE590E061
:103F00000E9442166DE671E084E690E00E9475160C
:103F10006BE671E087E690E00E94751667E771E056
:103F20008AE690E00E94751669E771E08DE690E000
:103F30000E9475166BE771E080E790E00E947516AD
:103F40006DE771E083E790E00E9475166FE771E01E
:103F500086E790E00E94751661E871E089E790E0DD
:103F60000E94751663E871E08CE790E00E94751678
:103F700065E871E08FE790E00E94751667E871E0F0
:103F800082E890E00E94751669E871E085E890E0AB
:103F90000E9475166BE871E088E890E00E94751643
:103FA0006DE871E08BE890E00E9475166FE871E0B3
:103FB0008EE890E00E94751661E971E081E990E079
:103FC0000E94751663E971E084E990E00E9475161D
:103FD00065E971E087E990E00E94751667E971E094
:103FE0008AE990E00E94751669E971E08DE990E038
:103FF0000E9475166BE971E080EA90E00E947516E8
:104000006DE971E083EA90E00E94751668E271E064
:104010008AEA90E00E94421664E271E08FEA90E042
:104020000E94421660E271E084EB90E00E9442162A
:104030006CE171E089EB90E00E94421668E171E06A
:104040008EEB90E00E94421664E171E083EC90E018
:104050000E94421660E171E088EC90E00E944216F6
:104060006CE071E08DEC90E00E94421668E071E037
:1040700082ED90E00E94421664EB71E090E080E0F7
:104080000E94EB13DC018C918093B40164E671E033
:1040900088E090E00E94EB13FC0180818093640132
:1040A0006FEA71E08DE090E00E94EB13DC018C91EF
:1040B0008093AF016AE175E08FE090E00E94FE120C
:1040C000FC0180819181A281B3818093B0019093A2
:1040D000B101A093B201B093B3016CE575E085E145
:1040E00090E00E94FE12FC0180819181A281B38147
:1040F0008093AB019093AC01A093AD01B093AE015E
:1041000063E771E08AE190E00E94FE12FC01808189
:104110009181A281B3818093730190937401A093E4
:104120007501B09376018FE190E00E947132809327
:10413000040180E290E00E9471328093050181E2E7
:1041400090E00E9471328093060182E290E00E942A
:104150007132809307018091040190910501A09133
:104160000601B09107018093B5019093B601A09329
:10417000B701B093B80160E375E084E290E00E947B
:10418000FE12FC0180819181A281B3818093A30101
:104190009093A401A093A501B093A6016FE671E0EE
:1041A00088E290E00E94FE12FC0180819181A28150
:1041B000B38180936F0190937001A0937101B093CC
:1041C000720169E671E087E390E00E94EA12DC0187
:1041D0008D919C9190936A018093690166E475E0EA
:1041E0008CE390E00E94FE12FC0180819181A2810B
:1041F000B3818093460590934705A0934805B093FB
:1042000049056FE971E08AE590E00E94FE12FC0129
:1042100080819181A281B38180939F019093A001BD
:10422000A093A101B093A2018091730190917401B8
:10423000A0917501B09176018093070790930807CC
:10424000A0930907B0930A07C0906F01D090700146
:10425000E0907101F09072010E94D20562E987EB53
:104260000E946507C114D104E104F104D9F08FE084
:104270000E94CA07682F6F73F1E8CF16F3ECDF06D0
:10428000F9ECEF06F1E0FF0610F00C948A29C092D9
:104290000D07D0920E07E0920F07F09210078FE003
:1042A0000E94650760E880E10E94650760E881E19F
:1042B0000E94650760E882E10E9465076CE080E18A
:1042C0000E9465076CE081E10E9465076CE082E175
:1042D0000E94650760E281EB0E94650760E881EB60
:1042E0000E94650710E000E020E03EE249E556E765
:1042F00061E170E080E090E00E94070D61E081E004
:1043000090E00E943E0890E080E00E94310881E049
:1043100090E00E94310882E090E00E9431086CE455
:1043200072E08AEC96E00E94771462E08EE00E94D0
:1043300004068091680084608093680080916D001D
:104340008C6080936D0078940E94A9066093160596
:1043500070931705809318059093190588EE93E0E4
:10436000A0E0B0E080931F0590932005A093210565
:10437000B09322058091640181110DC06EEC72E052
:1043800084EC96E00E94771481E080935A0561E006
:1043900080E10E94A40580916401813061F46EE4A3
:1043A00072E084EC96E00E94771410925A0560E067
:1043B00080E10E94A4058091290590912A0501972A
:1043C00009F097C080911F0590912005A0912105CB
:1043D000B091220585369105A105B105C0F08AE0AE
:1043E00090E0A0E0B0E08093650190936601A09317
:1043F0006701B09368012EE630E040E050E0209382
:104400001F0530932005409321055093220580918C
:104410001F0590912005A0912105B0912205899753
:10442000A109B109CC97A105B105C0F482E390E0E0
:10443000A0E0B0E08093650190936601A0936701CE
:10444000B093680126E430E040E050E020931F057F
:1044500030932005409321055093220580911F053C
:1044600090912005A0912105B09122054F97A109B7
:10447000B1090A97A105B105C0F484E690E0A0E077
:10448000B0E08093650190936601A0936701B093BB
:10449000680123E230E040E050E020931F053093B4
:1044A0002005409321055093220580911F0590918E
:1044B0002005A0912105B09122054F97A105B105D6
:1044C000C0F488EE93E0A0E0B0E0809365019093A3
:1044D0006601A0936701B09368012FE030E040E0EF
:1044E00050E020931F053093200540932105509301
:1044F00022058091720590917305892BC9F560E0C2
:1045000083E00E94AD098091B5019091B601A09120
:10451000B701B091B80180933A0590933B05A09301
:104520003C05B0933D056091B5017091B601809155
:10453000B7019091B80120E432E44FE050E00E94CE
:104540001434209336053093370540933805509343
:10455000390580E20E94DE090E94620A60E08FE075
:104560000E94AD096AEC76E081E197E00E94370491
:104570008EE00E9440068EE00E9440067C019093EF
:104580002805809327056AE070E080E090E00E94B3
:1045900077068EE00E9440068EE00E944006092EBB
:1045A000000CAA0BBB0BA7010F2C000C660B770BA2
:1045B0004C015D0133E0831A9108A108B108481548
:1045C00059056A057B0564F00396A11DB11D84178A
:1045D0009507A607B70724F0F0924505E092440539
:1045E000E0904405F090450545E8E41643E0F40604
:1045F0000CF4C9C61092260580912505811106C0CC
:1046000060E081E10E94A40510927105809169012A
:1046100090916A01009711F00C94102B21E030E08A
:1046200030932A052093290524EF31E040E050E043
:104630008530910511F00C94382B2093650130934F
:104640006601409367015093680110922A05109209
:1046500029058091720590917305181619060CF0C2
:10466000ADC3019701F560E080E00E94AD0986E5E9
:1046700092E00E94110B0E94130B61E084E00E9403
:10468000AD0987E494E00E94110B60917301709171
:10469000740180917501909176010E94380A86E735
:1046A00094E00E94110B809172059091730502971E
:1046B00089F560E080E00E94AD0988E692E00E9402
:1046C000110B0E94130B61E084E00E94AD09609120
:1046D000B0017091B1018091B2019091B3016093EA
:1046E0003A0570933B0580933C0590933D0520E48B
:1046F00032E44FE050E00E94363420933605309388
:10470000370540933805509339050E94620A80E2CC
:104710000E94DE098091720590917305039761F400
:104720000E94EA0A60E080E00E94AD0989E792E019
:104730000E94110B0E94130B8091720590917305DA
:10474000049759F50E94EA0A60E080E00E94AD09F2
:104750008AE892E00E94110B8091AF01811106C09E
:1047600064E472E084E996E00E9477148091AF01DE
:10477000813031F468E472E084E996E00E947714B5
:1047800061E080E00E94AD0964E976E081E197E0B4
:104790000E94370480E20E94DE09809172059091A8
:1047A0007305059709F04DC060E080E00E94AD09F7
:1047B0008BE992E00E94110B8091B401811106C037
:1047C00064E472E08AE996E00E9477148091B40173
:1047D000813031F468E472E08AE996E00E9477144F
:1047E00061E080E00E94AD096AE976E081E197E04E
:1047F0000E9437046091B0017091B1018091B201C3
:104800009091B30160933A0570933B0580933C050A
:1048100090933D0520E432E44FE050E00E943634AE
:10482000209336053093370540933805509339056A
:104830000E94620A88E494E00E94110B80E20E94C8
:10484000DE098091720590917305069709F560E085
:1048500080E00E94AD098CEA92E00E94110B61E0B9
:1048600080E00E94AD0982E594E00E94110B609106
:104870006F017091700180917101909172010E949D
:10488000380A8DEB92E00E94110B80E20E94DE0953
:104890008091720590917305079701F560E080E0C3
:1048A0000E94AD0981EC92E00E94110B0E94130B53
:1048B00061E084E00E94AD0987E494E00E94110B5E
:1048C00060913005709131058091320590913305EA
:1048D0000E94380A82ED92E00E94110B80917205CD
:1048E00090917305089719F560E080E00E94AD098A
:1048F0008AED92E00E94110B0E94130B61E084E0AC
:104900000E94AD0987E494E00E94110B60919F0121
:104910007091A0018091A1019091A2010E94380A9A
:1049200082ED92E00E94110B80E20E94DE098091EC
:104930007205909173050997F1F460E080E00E94A0
:10494000AD098BEE92E00E94110B87E494E00E9487
:10495000110B61E080E00E94AD098AE694E00E94BC
:10496000110B6EE876E081E197E00E9437048EE556
:1049700094E00E94110B80917205909173050A9743
:1049800009F01AC28091920690919306892B09F43E
:1049900013C2E0908E06F0908F0664E472E0C701C7
:1049A0000E94E037892B21F4109273051092720552
:1049B00068E472E0C7010E94E037892B09F0F2C178
:1049C0000E94A906C0905605D0905705E090580562
:1049D000F09059056C197D098E099F09653F71405A
:1049E0008105910508F4DEC161E080E00E94AD0917
:1049F0008CEF92E00E94110B60912C0570912D05B7
:104A000080912E0590912F0542E00E94730B8DE658
:104A100093E00E94110B80912B058130C1F40E941C
:104A2000A80760E080E00E94AD0988E093E00E9462
:104A3000110B809154059091550590936E018093D0
:104A40006D016DE671E084E690E00E94751680913C
:104A50002B058230D1F50E94A80760E080E00E941B
:104A6000AD098AE193E00E94110B80915405909169
:104A7000550590937A018093790120916D013091D1
:104A80006E01821B930B63E070E00E940034260FDE
:104A9000371F30936C0120936B01260F371F309323
:104AA0007801209377016BE671E087E690E00E9441
:104AB000751667E771E08AE690E00E94751669E76F
:104AC00071E08DE690E00E94751680912B05833091
:104AD000D1F50E94A80760E080E00E94AD098BE25A
:104AE00093E00E94110B809154059091550590938D
:104AF000800180937F012091790130917A01821B9E
:104B0000930B63E070E00E940034260F371F309350
:104B10007C0120937B01260F371F30937E01209369
:104B20007D016BE771E080E790E00E9475166DE70C
:104B300071E083E790E00E9475166FE771E086E709
:104B400090E00E94751680912B058430D1F50E946B
:104B5000A80760E080E00E94AD098CE393E00E942A
:104B6000110B809154059091550590938601809387
:104B7000850120917F0130918001821B930B63E0BE
:104B800070E00E940034260F371F3093820120937B
:104B90008101260F371F309384012093830161E840
:104BA00071E089E790E00E94751663E871E08CE798
:104BB00090E00E94751665E871E08FE790E00E9432
:104BC000751680912B05853009F048C00E94A80712
:104BD00060E080E00E94AD098DE493E00E94110B3B
:104BE000809154059091550590938E0180938D018D
:104BF0002091850130918601821B930B97FD0396CE
:104C00009595879595958795280F391F309388013D
:104C100020938701280F391F30938A01209389013F
:104C2000820F931F90938C0180938B0167E871E052
:104C300082E890E00E94751669E871E085E890E0EE
:104C40000E9475166BE871E088E890E00E94751686
:104C50006DE871E08BE890E00E94751680912B055D
:104C6000863009F048C00E94A80760E080E00E94FA
:104C7000AD098EE593E00E94110B8091540590914F
:104C80005505909396018093950120918D01309167
:104C90008E01821B930B97FD0396959587959595AD
:104CA0008795280F391F3093900120938F01280F8B
:104CB000391F3093920120939101820F931F90939B
:104CC0009401809393016FE871E08EE890E00E9478
:104CD000751661E971E081E990E00E94751663E95B
:104CE00071E084E990E00E94751665E971E087E95A
:104CF00090E00E94751680912B05873009F048C01E
:104D00000E94A80760E080E00E94AD098FE693E072
:104D10000E94110B809154059091550590939E012E
:104D200080939D012091950130919601821B930BF8
:104D300097FD03969595879595958795280F391F2B
:104D40003093980120939701280F391F30939A01CF
:104D500020939901820F931F90939C0180939B0154
:104D600067E971E08AE990E00E94751669E971E0EF
:104D70008DE990E00E9475166BE971E080EA90E0A1
:104D80000E9475166DE971E083EA90E00E94751645
:104D90000E94A906609356057093570580935805A5
:104DA0009093590580917205909173050B9724F0AB
:104DB00010927305109272050E94D41480917105AF
:104DC0008130B9F58091720590917305892B89F531
:104DD000E0903405F0903505BFEFEB1AFB0AF09236
:104DE0003505E092340584E10E944006BC01990F2C
:104DF000880B990B0E9454312B013C0185E10E94E4
:104E00004006BC01990F880B990B0E9454314B014D
:104E10005C01AC019B01C301B2010E94E63387FD36
:104E200067C461E080E00E94AD0980E893E00E94E1
:104E3000110B81E090917005913009F080E091E0D4
:104E400020917105211190E0892309F4BFC0809160
:104E5000720590917305892B09F0B8C08091A70164
:104E60009091A801A091A901B091AA018032F1EA24
:104E70009F07F7E0AF07B1050CF0CBC48091B501F7
:104E80009091B601A091B701B091B8018052914ABA
:104E9000A740B109B095A095909581959F4FAF4FD0
:104EA000BF4F8093460590934705A0934805B09364
:104EB0004905809144059091450587599109C1970D
:104EC000D0F48091420590914305843691059CF47D
:104ED00001969093430580934205C29761F4109226
:104EE0004605109247051092480510924905109208
:104EF0004305109242050E94130B8091B5019091D9
:104F0000B601A091B701B091B8014091460550910A
:104F100047056091480570914905840F951FA61FAC
:104F2000B71F8093A7019093A801A093A901B09304
:104F3000AA0180913E0590913F05A0914005B09156
:104F40004105481759076A077B07B1F066E475E029
:104F50008CE390E00E9442168091460590914705AF
:104F6000A0914805B091490580933E0590933F0577
:104F7000A0934005B093410561E084E00E94AD0933
:104F80006091A7017091A8018091A9019091AA0157
:104F900060933A0570933B0580933C0590933D05E3
:104FA00020E432E44FE050E00E943634209336058E
:104FB0003093370540933805509339050E94620AB3
:104FC00080E20E94DE0980E20E94DE098091710584
:104FD00090917005892B09F0FCC080917205909129
:104FE0007305892B09F0F5C069E474E08CEA96E05A
:104FF0000E9477140E94A8070E94A9060E94A90691
:10500000C0905605D0905705E0905805F09059058E
:105010006C197D098E099F0964367105810591051A
:1050200040F48091540590915505909353058093D9
:1050300052050E94A9066C197D098E099F096436E4
:1050400071058105910598F00E94A9066C197D09EA
:105050008E099F09683C71058105910540F4809196
:1050600054059091550590935105809350050E94E9
:10507000A9066C197D098E099F09683C7105810597
:10508000910598F00E94A9066C197D098E099F0967
:105090006C3271408105910540F4809154059091E6
:1050A000550590934F0580934E050E94A9066C19F3
:1050B0007D098E099F096C3271408105910598F038
:1050C0000E94A9066C197D098E099F0960397140FB
:1050D0008105910540F48091540590915505909378
:1050E0004D0580934C050E94A9066C197D098E0917
:1050F0009F09603971408105910598F00E94A906C9
:105100006C197D098E099F09653F714081059105E4
:1051100040F4809154059091550590934B058093F0
:105120004A050E94A9066C197D098E099F09653FF1
:1051300071408105910508F44AC080915205909113
:1051400053052091500530915105820F931F2091F6
:105150004E0530914F05820F931F20914C053091E1
:105160004D05820F931F20914A0530914B05820F08
:10517000931F65E070E00E9400347B017093550539
:10518000609354056DE971E083EA90E00E94EA12B1
:10519000DC018D919C91E816F9060CF451C381EA6B
:1051A00093E00E94491461E084E00E94AD096CEA3A
:1051B00076E081E197E00E9437040E94A90660939F
:1051C00056057093570580935805909359050E9492
:1051D000130B6CE575E085E190E00E94FE12FC0186
:1051E00080819181A281B3818093AB019093AC01C6
:1051F000A093AD01B093AE0110917105113081F40F
:105200008091B5019091B601A091B701B091B8011C
:105210008093A7019093A801A093A901B093AA013C
:105220008091B5019091B601A091B701B091B801FC
:1052300080389F49A54DB10508F412C580915B05E2
:1052400081113EC46CE472E08AEC96E00E9477140F
:1052500062E572E08EEB96E00E9477148091700513
:10526000813009F022C48091A7019091A801A091FA
:10527000A901B091AA014091B0015091B101609192
:10528000B2017091B301841B950BA60BB70B409133
:10529000AB015091AC016091AD017091AE01841BE6
:1052A000950BA60BB70B80936C0590936D05A0939F
:1052B0006E05B0936F0580915A05813009F072C474
:1052C000113009F06FC480916C0590916D05A0912B
:1052D0006E05B0916F054091A3015091A4016091BA
:1052E000A5017091A601841B950BA60BB70B52C4A8
:1052F0008EE00E944006853F914014F40C943C20BF
:105300008EE00E9440068A38924014F40C94371FB5
:105310000C943C20D701C6018158934CA94CB14054
:105320008038934CA94CB14078F4F694E794D79424
:10533000C794C0920D07D0920E07E0920F07F0922B
:10534000100760640C944F21D701C6018150974823
:10535000A349B34081159A45A246B24010F00C947F
:105360004F2172E0F694E794D794C7947A95D1F7D9
:10537000C0920D07D0920E07E0920F07F09210072F
:1053800060680C944F2158E4E516F1046CF48091A8
:105390002605811109C061E081E10E94A40581E038
:1053A0008093710580932605C701895491098D3436
:1053B000910538F580912605811123C0809125053E
:1053C00081110BC061E081E10E94A40581E080931E
:1053D000250580937105809326058091260581110E
:1053E00015C910912505113009F010C960E081E15F
:1053F0000E94A405109225051092710510932605B0
:1054000005C9C701875991098034910508F5809134
:10541000260581111DC080917005811109C081E0B0
:1054200080937005809326051092430510924205E3
:105430008091260581110CC080917005813041F466
:105440001092700580932605109243051092420534
:10545000C701885D9109C697C8F48091260581111E
:1054600015C08091230590912405019688309105FF
:1054700054F4909324058093230581E080932605BE
:105480000E942413C3C888E090E0F3CFC7018F5077
:105490009140C19788F48091260581110DC08091BB
:1054A00023059091240501971816190614F31092FC
:1054B000240510922305E1CFC701815491408C97B8
:1054C000C0F580912605811134C080915A05811163
:1054D00011C061E080E10E94A405109264016EECAD
:1054E00072E084EC96E00E94771481E080935A0584
:1054F0008093260580912605811114C010915A05CC
:10550000113081F460E080E10E94A40510936401F1
:105510006EE472E084EC96E00E94771410925A05D3
:105520001093260564E671E088E090E00E949C16E6
:105530006DC8C7018E5691408297D8F48091260598
:10554000811117C080915B05811105C081E08093B6
:105550005B058093260580912605811157C88091AF
:105560005B05813009F052C810925B0580932605D7
:105570004DC88091690190916A019701215931408C
:1055800022323105C8F420912605211115C001965B
:105590008830910574F490936A018093690181E0E9
:1055A0008093260569E671E087E390E00E94751616
:1055B0002DC888E090E0EFCF97012F5A3140233675
:1055C000310568F420912605211109C001971816AC
:1055D00019060CF310926A0110926901E0CF83E181
:1055E000E81A82E0F80A97E7E916F10408F00EC815
:1055F0008091260581110AC88091720590917305EA
:105600000196909373058093720521E020932B05FA
:105610000A9724F0109273051092720581E0A6CFCC
:105620008130910591F421E030E040E050E020939A
:1056300065013093660140936701509368011092B1
:105640002A05109229050C94142382309105C1F487
:105650002AE030E040E050E020936501309366019D
:10566000409367015093680110922A051092290512
:1056700086309105C1F488EE93E0A0E0B0E025C04B
:1056800083309105C9F422E330E040E050E02093FC
:105690006501309366014093670150936801109251
:1056A0002A051092290587309105C9F420E137E2D7
:1056B00040E050E00C941D238430910511F00C94CF
:1056C000142384E690E0A0E0B0E08093650190931D
:1056D0006601A0936701B09368010C942523089795
:1056E00011F00C94292380EA96E8A1E0B0E0EDCF18
:1056F000E4E1EE16F1040CF49CCB10923505109207
:105700003405A5019401C301B2010E94D9326B0195
:105710007C01A3019201C501B4010E94D8329B0112
:10572000AC01C701B6010E9445336B017C0120E04A
:1057300030E0A9010E94E633181624F0F7FAF0943D
:10574000F7F8F09420E030E040EA50E4C501B401FD
:105750000E94B33120E030EC4FE754E40E9445331F
:105760002CE238E540EB5CE30E9445339B01AC0141
:105770000E94B33120E030E048E452E40E94453317
:105780004B015C0120E030E040E050E4C701B6018D
:105790000E94D9322B013C01A701960160E070E024
:1057A00080E89FE30E9445339B01AC01C301B20135
:1057B0000E94D9329B01AC0160E070E080E890E487
:1057C0000E944533A50194010E94B3314B015C0155
:1057D00061E080E00E94AD0983E993E00E94110B33
:1057E00042E0C701B6010E94730B61E088E00E94AD
:1057F000AD0988E993E00E94110B61E08BE00E9403
:10580000AD0940E0C501B4010E94730B8CE993E03F
:105810000ECB8130914EA54FB5400CF44ACB409150
:10582000B5015091B6016091B7017091B80180E067
:1058300091EEA5EFB5E0841B950BA60BB70B31CB12
:105840006DE971E083EA90E00E94EA12FC01808138
:1058500091818E159F051CF48EEA93E0A2CC6BE932
:1058600071E080EA90E00E94EA12DC018D919C9147
:105870008E159F051CF48BEB93E093CC69E971E0E6
:105880008DE990E00E94EA12FC01808191818E15E1
:105890009F051CF488EC93E084CC67E971E08AE909
:1058A00090E00E94EA12DC018D919C918E159F057B
:1058B0001CF485ED93E075CC65E971E087E990E033
:1058C0000E94EA12FC01808191818E159F051CF4D3
:1058D00082EE93E066CC63E971E084E990E00E9497
:1058E000EA12DC018D919C918E159F051CF48FEEC0
:1058F00093E057CC61E971E081E990E00E94EA12FF
:10590000FC01808191818E159F051CF48CEF93E042
:1059100048CC6FE871E08EE890E00E94EA12DC016A
:105920008D919C918E159F051CF489E094E039CCF3
:105930006DE871E08BE890E00E94EA12FC01808142
:1059400091818E159F051CF486E194E02ACC6BE8CA
:1059500071E088E890E00E94EA12DC018D919C9150
:105960008E159F051CF483E294E01BCC69E871E07E
:1059700085E890E00E94EA12FC01808191818E15F9
:105980009F051CF480E394E00CCC67E871E082E8AA
:1059900090E00E94EA12DC018D919C918E159F058A
:1059A0001CF48DE394E0FDCB65E871E08FE790E0B7
:1059B0000E94EA12FC01808191818E159F051CF4E2
:1059C0008AE494E0EECB63E871E08CE790E00E941B
:1059D000EA12DC018D919C918E159F051CF487E5E0
:1059E00094E0DFCB61E871E089E790E00E94EA1281
:1059F000FC01808191818E159F051CF484E694E062
:105A0000D0CB6FE771E086E790E00E94EA12DC01FC
:105A10008D919C918E159F051CF481E794E0C1CB7C
:105A20006DE771E083E790E00E94EA12FC0180815B
:105A300091818E159F051CF48EE794E0B2CB6BE745
:105A400071E080E790E00E94EA12DC018D919C9168
:105A50008E159F051CF48BE894E0A3CB69E771E0F9
:105A60008DE690E00E94EA12FC01808191818E1502
:105A70009F051CF488E994E094CB67E771E08AE61F
:105A800090E00E94EA12DC018D919C918E159F0599
:105A90001CF485EA94E085CB67E771E087E690E047
:105AA0000E94EA1282EB94E07CCB811104CC8091BD
:105AB000B5019091B601A091B701B091B801DBCBCF
:105AC000813009F0CDC06FEB74E08AEC96E00E9463
:105AD000771461EC74E08EEB96E00E94771480916D
:105AE0007005813009F0A9C04091AB015091AC0123
:105AF0006091AD017091AE018091A7019091A801D4
:105B0000A091A901B091AA01C090B001D090B101BB
:105B1000E090B201F090B3018C199D09AE09BF0964
:105B2000841B950BA60BB70B80936C0590936D05AA
:105B3000A0936E05B0936F0580919F019091A00195
:105B4000A091A101B091A201840F951FA61FB71FBC
:105B50008093AB019093AC01A093AD01B093AE01E3
:105B600080915A058130F1F41130E1F480916C0597
:105B700090916D05A0916E05B0916F054091A301C4
:105B80005091A4016091A5017091A601840F951F09
:105B9000A61FB71F80936C0590936D05A0936E05AB
:105BA000B0936F058091B401811105C060E081E080
:105BB00090E00E943E088091B401813009F0F7C165
:105BC00061E081E090E00E943E0840916C055091B8
:105BD0006D0560916E0570916F05809168059091DB
:105BE0006905A0916A05B0916B05481759076A07C6
:105BF0007B0709F0BAC12091C2063091C30680919B
:105C0000BC069091BD062817390709F0AEC18091F6
:105C1000BE069091BF066091B8067091B9060097D4
:105C200009F496C16115710509F0F3C0232B09F43D
:105C3000BEC1FC01808190E096C1811191CF80911D
:105C4000B5019091B601A091B701B091B801409112
:105C5000AB015091AC016091AD017091AE0154CF98
:105C60008091B5019091B601A091B701B091B801B2
:105C700080389F49A54DB10508F094CF80915B0510
:105C8000811158C06FEB74E08AEC96E00E947714A3
:105C900062E572E08EEB96E00E94771480917005C9
:105CA000813049F58091A7019091A801A091A901A7
:105CB000B091AA014091B0015091B1016091B2013F
:105CC0007091B301840F951FA61FB71F4091AB01C0
:105CD0005091AC016091AD017091AE01840F951FA0
:105CE000A61FB71F80936C0590936D05A0936E055A
:105CF000B0936F0535CF811133CF4091B5015091ED
:105D0000B6016091B7017091B8018091B001909196
:105D1000B101A091B201B091B301C090AB01D0909C
:105D2000AC01E090AD01F090AE018C0D9D1DAE1D5B
:105D3000BF1DD4CF813009F035CF6CE472E08AEC1E
:105D400096E00E94771461EC74E08EEB96E00E947E
:105D50007714809170058130E9F54091AB01509145
:105D6000AC016091AD017091AE018091A70190915D
:105D7000A801A091A901B091AA01840F951FA61FA7
:105D8000B71FC090B001D090B101E090B201F09087
:105D9000B3018C0D9D1DAE1DBF1D80936C059093AE
:105DA0006D05A0936E05B0936F0580919F01909152
:105DB000A001A091A101B091A201840F951FA61F7F
:105DC000B71F8093AB019093AC01A093AD01B0934A
:105DD000AE0171CA81116FCAC090B501D090B601F1
:105DE000E090B701F090B8014091AB015091AC0147
:105DF0006091AD017091AE018091B0019091B101BF
:105E0000A091B201B091B301840F951FA61FB71FD7
:105E1000C0CF0E94E037A7C088EB96E00E94D31263
:105E2000C6C00E9491368AA19BA19093A10680933F
:105E3000A0068CA19DA19093A3068093A2068EA19B
:105E40009FA19093A5068093A4061BA21AA21DA24F
:105E50001CA25BC180EA96E00E94D31296C165EC59
:105E600074E0CE0101960E9481144091A4065091E5
:105E7000A5066091A0067091A106CE0101960E9430
:105E80001D14811104C0CE0101960E94D31241E07D
:105E900050E068EC74E0CE0101960E941D1481115F
:105EA00004C0CE0101960E94D312BE016F5F7F4FE6
:105EB00085EE95E00E943704CE0101960E94E5121E
:105EC00064E170E080E090E00E9477060E94D414C4
:105ED00080916C0590916D05A0916E05B0916F0554
:105EE0008093680590936905A0936A05B0936B054C
:105EF0008091B5019091B601A091B701B091B80120
:105F00008093600590936105A0936205B09363054B
:105F10008091720590917305892B51F460E080E0C7
:105F20000E94AD0964EC76E081E197E00E943704BD
:105F300080E090E0892B11F40C94DB210E94AF04E7
:105F4000882311F40C94DB210E9400000C94DB21C7
:105F50006115710561F1232B51F1DB018C9190E00A
:105F6000919581959109892B11F16091B001709102
:105F7000B1018091B2019091B30124E630E040E09C
:105F800050E00E94AD3401E010E00E94B70E609135
:105F9000BE067091BF066115710509F43DCF4091B1
:105FA000C2065091C30688EB96E00E945614809179
:105FB000AF01811105C060E082E090E00E943E08E0
:105FC0008091AF018130A1F561E082E090E00E9414
:105FD0003E086091AB017091AC018091AD01909150
:105FE000AE01C0906405D0906505E0906605F09024
:105FF00067056C157D058E059F05D1F024E630E020
:1060000040E050E00E94AD3402E010E00E94B70E84
:106010008091AB019091AC01A091AD01B091AE0126
:106020008093640590936505A0936605B09367051A
:1060300040916C0550916D0560916E0570916F05F2
:106040008091680590916905A0916A05B0916B05F2
:10605000481759076A077B0709F45ACF80917205E0
:1060600090917305892B09F053CF60916C05709165
:106070006D0580916E0590916F0524E630E040E05B
:1060800050E00E94BC3410E000E00E94B70E8FE1A7
:1060900090E00E94AB146091B5017091B6018091BF
:1060A000B7019091B8011BA21AA21DA21CA21FA2A7
:1060B0001EA22AE0AE014F5F5F4F0E940131BE0178
:1060C0006F5F7F4FCE0182960E9477148091A00669
:1060D0009091A106009709F4A6CE6AA17BA1611553
:1060E000710509F49ECE4091A2065091A3062EA1FF
:1060F0003FA14217530708F494CE0E94E9378EA1BE
:106100009FA19093A5068093A4061FA21EA2CE0174
:1061100082960E94E5128091A4069091A5060B97A5
:1061200008F09DCE1BA21AA21DA21CA21FA21EA295
:106130004AE0BE016F5F7F4F90E080E00E94F63042
:10614000BE016F5F7F4FCE0182960E94771440910F
:10615000A4065091A5066091A0067091A106CE01FB
:1061600082960E941D14811104C0CE0182960E9465
:10617000D3126AA17BA16115710509F46BCE4EA102
:106180005FA180EA96E00E945614CE0182960E949A
:10619000E512C1CF8EE896E00E94E51284E996E010
:1061A0000E94E5128AE996E00E94E51280EA96E0F4
:1061B0000E94E51286EA96E00E94E5128CEA96E0DB
:1061C0000E94E51282EB96E00E94E51288EB96E0D1
:1061D0000E94E5128EEB96E00E94E51284EC96E0B8
:1061E0000E94E5128AEC96E00C94E512BB274A3037
:1061F00031F4992322F4BDE2909581959F4F0C9440
:106200002431BB27FA01A62F62177105810591057C
:10621000330B30FB66F0AA27660F771F881F991F84
:10622000AA1FA21710F0A21B63953850A9F7A05D12
:10623000AA3308F0A95DA19336F7B111B19310828A
:10624000CA010C943D31BB27FB015527AA27880FB3
:10625000991FAA1FA41710F0A41B83955051B9F7DA
:10626000A05DAA3308F0A95DA193009779F7B11159
:10627000B1931192CB010C943D31DC01FC01672FED
:1062800071917723E1F7329704C07C916D9370830D
:106290006291AE17BF07C8F308950E948F3108F4CA
:1062A00081E00895E89409C097FB3EF490958095AD
:1062B000709561957F4F8F4F9F4F9923A9F0F92FCC
:1062C00096E9BB279395F695879577956795B7954A
:1062D000F111F8CFFAF4BB0F11F460FF1BC06F5F30
:1062E0007F4F8F4F9F4F16C0882311F096E911C042
:1062F000772321F09EE8872F762F05C0662371F063
:1063000096E8862F70E060E02AF09A95660F771F76
:10631000881FDAF7880F9695879597F90895990F52
:106320000008550FAA0BE0E8FEEF16161706E8075F
:10633000F907C0F012161306E407F50798F0621B80
:10634000730B840B950B39F40A2661F0232B242B55
:10635000252B21F408950A2609F4A140A6958FEF74
:10636000811D811D08950E94C6310C9437320E9410
:10637000293238F00E94303220F0952311F00C942D
:1063800020320C94263211240C946B320E94483235
:1063900070F3959FC1F3950F50E0551F629FF00178
:1063A000729FBB27F00DB11D639FAA27F00DB11D91
:1063B000AA1F649F6627B00DA11D661F829F22271A
:1063C000B00DA11D621F739FB00DA11D621F839FA1
:1063D000A00D611D221F749F3327A00D611D231F77
:1063E000849F600D211D822F762F6A2F11249F57C5
:1063F00050409AF0F1F088234AF0EE0FFF1FBB1FC8
:10640000661F771F881F91505040A9F79E3F510586
:1064100080F00C9420320C946B325F3FE4F3983E92
:10642000D4F3869577956795B795F795E7959F5F30
:10643000C1F7FE2B880F911D9695879597F90895C2
:1064400097F99F6780E870E060E008959FEF80EC27
:10645000089500240A9416161706180609060895CA
:1064600000240A9412161306140605060895092E30
:106470000394000C11F4882352F0BB0F40F4BF2B9F
:1064800011F460FF04C06F5F7F4F8F4F9F4F0895DF
:1064900057FD9058440F551F59F05F3F71F04795D5
:1064A000880F97FB991F61F09F3F79F087950895BA
:1064B000121613061406551FF2CF4695F1DF08C0D9
:1064C000161617061806991FF1CF869571056105F6
:1064D00008940895E894BB2766277727CB0197F99E
:1064E0000895F999FECF92BD81BDF89A992780B59C
:1064F0000895262FF999FECF1FBA92BD81BD20BD08
:106500000FB6F894FA9AF99A0FBE019608950E9470
:10651000C932A59F900DB49F900DA49F800D911D31
:10652000112408952F923F924F925F926F927F9223
:106530008F929F92AF92BF92CF92DF92EF92FF9293
:106540000F931F93CF93DF93CDB7DEB7CA1BDB0B3F
:106550000FB6F894DEBF0FBECDBF09942A883988E4
:1065600048885F846E847D848C849B84AA84B984EB
:10657000C884DF80EE80FD800C811B81AA81B981F7
:10658000CE0FD11D0FB6F894DEBF0FBECDBFED010B
:106590000895A29FB001B39FC001A39F700D811DFC
:1065A0001124911DB29F700D811D1124911D08951C
:1065B0005058BB27AA270E94F0320C9437320E9411
:1065C000293238F00E94303220F039F49F3F19F41C
:1065D00026F40C9426320EF4E095E7FB0C9420325E
:1065E000E92F0E94483258F3BA17620773078407ED
:1065F000950720F079F4A6F50C946A320EF4E09534
:106600000B2EBA2FA02D0B01B90190010C01CA016C
:10661000A0011124FF27591B99F0593F50F4503E17
:1066200068F11A16F040A22F232F342F4427585F09
:10663000F3CF469537952795A795F0405395C9F721
:106640007EF41F16BA0B620B730B840BBAF09150D9
:10665000A1F0FF0FBB1F661F771F881FC2F70EC078
:10666000BA0F621F731F841F48F48795779567954B
:10667000B795F7959E3F08F0B0CF9395880F08F037
:106680009927EE0F9795879508950E9459330C949A
:1066900037320E94303258F00E94293240F029F4FB
:1066A0005F3F29F00C94203251110C946B320C9402
:1066B00026320E94483268F39923B1F3552391F3AF
:1066C000951B550BBB27AA2762177307840738F061
:1066D0009F5F5F4F220F331F441FAA1FA9F335D0BE
:1066E0000E2E3AF0E0E832D091505040E695001C72
:1066F000CAF72BD0FE2F29D0660F771F881FBB1F2C
:10670000261737074807AB07B0E809F0BB0B802D09
:10671000BF01FF2793585F4F3AF09E3F510578F035
:106720000C9420320C946B325F3FE4F3983ED4F328
:10673000869577956795B795F7959F5FC9F7880F09
:10674000911D9695879597F90895E1E0660F771F5B
:10675000881FBB1F621773078407BA0720F0621BEC
:10676000730B840BBA0BEE1F88F7E09508950E9417
:10677000503288F09F5798F0B92F9927B751B0F051
:10678000E1F0660F771F881F991F1AF0BA95C9F7B5
:1067900014C0B13091F00E946A32B1E008950C94B7
:1067A0006A32672F782F8827B85F39F0B93FCCF36A
:1067B000869577956795B395D9F73EF49095809532
:1067C000709561957F4F8F4F9F4F08950E948F3135
:1067D00008F48FEF08950E948F31880B990B08956C
:1067E000DB018F939F930E948732BF91AF91A29F4D
:1067F000800D911DA39F900DB29F900D11240895BF
:1068000097FB072E16F4009407D077FD09D00E945D
:10681000DB3507FC05D03EF4909581959F4F089598
:10682000709561957F4F0895A1E21A2EAA1BBB1B9C
:10683000FD010DC0AA1FBB1FEE1FFF1FA217B3074C
:10684000E407F50720F0A21BB30BE40BF50B661F62
:10685000771F881F991F1A9469F760957095809526
:1068600090959B01AC01BD01CF010895052E97FBCA
:106870001EF400940E944D3457FD07D00E9414343A
:1068800007FC03D04EF40C944D3450954095309550
:1068900021953F4F4F4F5F4F08959095809570958C
:1068A00061957F4F8F4F9F4F0895DF93CF931F9335
:1068B0000F939A9DF02D219FF00D8B9DF00D8A9DD9
:1068C000E02DF10D039FF00D029FE00DF11D4E9D97
:1068D000E00DF11D5E9DF00D4F9DF00D7F936F93C8
:1068E000BF92AF925F934F93D5010E94C9328B0143
:1068F000AC01D7010E94C932EB01E80FF91FD601A4
:106900000E94A4342F913F91D6010E94C932C60F34
:10691000D71FE81FF91FAF91BF910E94A4342F9198
:106920003F910E94C932C60FD71FE81FF91FD60139
:106930000E94C932E60FF71F9801BE01CF010F91E7
:106940001F91CF91DF9108950E94C932460F571FC2
:10695000C81FD91F08F43196089597FB57FF0C9470
:10696000BD349F938F930E94BD346E1B7F0BAF91FC
:10697000BF918A0B9B0B0895E894DF93CF93FC01A2
:10698000DB010E94C9327F936F93E9019A01AC0148
:10699000BF93AF933F932F93DF010E94C93226F438
:1069A0006C1B7D0B820B930B9E01EB01FC010E9483
:1069B000A434AF91BF912F913F910E94A434BE01A6
:1069C000CF01F9012F913F91CF91DF910895689404
:1069D00001C0E894F92FF12B12F00C941B35A0E0C4
:1069E000B0E0E5EFF4E30C949832092E059422F41C
:1069F0000E947735112392F4F0E80F26FFEFE09420
:106A0000F09400951095B094C094D094A194BF0ACE
:106A1000CF0ADF0AEF0AFF0A0F0B1F0B0E94263571
:106A200007FC0E947735CDB7DEB7ECE00C94B432AA
:106A3000689401C0E8948F929F92CF93DF930E9455
:106A40002635DF91CF919F908F90089588249924C7
:106A5000F401E401B0E49F93AA279A158B049C04E7
:106A6000ED05FE05CF05D007A10798F4AD2FDC2F6B
:106A7000CF2FFE2FE92D982C892E982F872F762F38
:106A8000652F542F432F322F2227B85031F7BF9153
:106A900027C01B2EBF91BB27220F331F441F551F3A
:106AA000661F771F881F991F881C991CEE1FFF1FE8
:106AB000CC1FDD1FAA1FBB1F8A149B04EC05FD051C
:106AC000CE05DF05A007B10748F08A189B08EC093E
:106AD000FD09CE09DF09A00BB10B21601A94E1F684
:106AE0002EF49401AF01BE01CD01000C0895609514
:106AF00070958095909530954095509521953F4F94
:106B00004F4F5F4F6F4F7F4F8F4F9F4F0895002E16
:106B1000083090F0982F872F762F652F542F432F12
:106B2000322F22270850F4CF220F331F441F551F46
:106B3000661F771F881F991F0A95B2F7002D0895C9
:106B400097FD1094002E083098F00850232F342F12
:106B5000452F562F672F782F892F912DF4CF15941D
:106B60009795879577956795579547953795279585
:106B70000A95AAF71124002D08952A0D3B1D4C1DDE
:106B80005D1D6E1D7F1D801F911F08952A153B05F9
:106B90004C055D056E057F0580079107089500246B
:106BA000A7FD00942A1730054005500560057005C3
:106BB000800590050895AA1BBB1B51E107C0AA1FC1
:106BC000BB1FA617B70710F0A61BB70B881F991F8E
:106BD0005A95A9F780959095BC01CD010895EE0FC7
:106BE000FF1F0590F491E02D09940F931F93CF930D
:106BF000DF938230910510F482E090E0E0912B0762
:106C0000F0912C0730E020E0B0E0A0E0309799F45C
:106C10002115310509F44AC0281B390B24303105F0
:106C2000D8F58A819B816115710589F1FB019383F8
:106C30008283FE0111C04081518102811381481776
:106C40005907E0F04817590799F4109761F0129628
:106C50000C93129713961C933296CF01DF91CF912C
:106C60001F910F91089500932B0710932C07F4CFD9
:106C70002115310551F04217530738F0A901DB0106
:106C80009A01BD01DF01F801C1CFEF01F9CF909367
:106C90002C0780932B07CDCFFE01E20FF31F8193CA
:106CA00091932250310939832883D7CF2091290726
:106CB00030912A07232B41F42091BB013091BC0174
:106CC00030932A07209329072091B9013091BA0106
:106CD0002115310541F42DB73EB74091BD015091CA
:106CE000BE01241B350BE0912907F0912A07E2171A
:106CF000F307A0F42E1B3F0B2817390778F0AC01DF
:106D00004E5F5F4F2417350748F04E0F5F1F5093BB
:106D10002A0740932907819391939FCFF0E0E0E009
:106D20009CCFCF93DF930097E9F0FC013297138259
:106D30001282A0912B07B0912C07ED0130E020E0EA
:106D40001097A1F420813181820F931F2091290790
:106D500030912A072817390709F061C0F0932A07F4
:106D6000E0932907DF91CF910895EA01CE17DF075D
:106D7000E8F54A815B819E0141155105B1F7E901B2
:106D8000FB83EA8349915991C40FD51FEC17FD0786
:106D900061F4808191810296840F951FE9019983A6
:106DA0008883828193819B838A83F0E0E0E012965E
:106DB0008D919C9113970097B9F52D913C91119766
:106DC000CD010296820F931F2091290730912A0747
:106DD0002817390739F6309751F510922C07109281
:106DE0002B07B0932A07A0932907BCCFD383C28374
:106DF00040815181840F951FC817D90761F44E5FF8
:106E00005F4F88819981480F591F518340838A8140
:106E10009B81938382832115310509F0B0CFF093D4
:106E20002C07E0932B079ECFFD01DC01C0CF13821E
:106E30001282D7CFB0E0A0E0E0E2F7E30C94943206
:106E40008C01009751F4CB010E94F5358C01C801EB
:106E5000CDB7DEB7E0E10C94B032FC01E60FF71FCE
:106E60009C0122503109E217F30708F49DC0D901B3
:106E7000CD91DC911197C617D70798F0C530D10591
:106E800030F3CE0104978617970708F3C61BD70B7C
:106E90002297C193D1936D937C93CF010E94913639
:106EA000D6CF5B01AC1ABD0A4C018C0E9D1EA09181
:106EB0002B07B0912C07512C412CF12CE12C109771
:106EC00031F58091290790912A078815990509F0D5
:106ED0005CC04616570608F058C08091B9019091E1
:106EE000BA01009741F48DB79EB74091BD01509112
:106EF000BE01841B950BE817F90708F055C0F09305
:106F00002A07E0932907F90171836083A0CF8D914F
:106F10009C91119712966C90129713967C901397F0
:106F2000A815B90559F56C0142E0C40ED11CCA146C
:106F3000DB0420F1AC014A195B09DA0112961597BE
:106F400080F06282738251834083D9016D937C9378
:106F5000E114F10471F0D7011396FC93EE931297AC
:106F600076CF22968C0F9D1FF90191838083F301C8
:106F7000EFCFF0932C07E0932B0769CF4816590603
:106F800008F42C017D01D3019ACFCB010E94F53585
:106F90007C01009749F0AE01B8010E94D737C801C3
:106FA0000E949136870153CF10E000E050CFFB01E3
:106FB000DC0102C001900D9241505040D8F7089575
:106FC000FB01DC018D91019080190110D9F3990B1F
:106FD0000895FB01DC0101900D920020E1F7089576
:106FE00010E0C2E6D0E004C0FE010E94EF35219619
:0A6FF000C336D107C9F7F894FFCFAC
:106FFA00C0320A03B0196D0020E0B201903B7E0155
:10700A00D03F4401407D140170E9D700406B9A00DB
:10701A0010936B00D0B13700903A1C001F11151164
:10702A001D1D111F1F1115111515111F1F111D1DD2
:10703A001D1D1D1F1F1117111515111F1F111711C6
:10704A001D1D111F1F1515111D1D1D1F1F111D119E
:10705A001D1D111F0132000000030079003C004091
:10706A00787D01CCF803009301BE01EA01FE01120A
:10707A000226023A026C02BA02E4020C0348035CDA
:10708A0003720388039D03A103A403A803AC03B8F6
:10709A000B0000A8FDFFFF40420F0020A1070001DE
:1070AA0060EC53000170E9D70000002D0780000052
:1070BA00020400030001100302000003020100069B
:1070CA00000400060500200605040000000000E593
:1070DA0004450472043205A30481049504000000E7
:1070EA000036070907A507E606EA00F606E70600DE
:1070FA00000000BC094504A507360431487A20007F
:10710A003130487A003530487A003130304800351D
:10711A0030304800316B487A0031306B48003130EA
:10712A00306B004175746F006E616E00696E6600A7
:10713A006F7666004F6666004F6E20005500535307
:10714A0042004C534200436F72722E504C4C2053F3
:10715A006935333531202000436F72722E20467212
:10716A0065712042464F2D3100436F72722E2046C0
:10717A007265712042464F2D320020202020204384
:10718A004C4B202D2032202020200020202020209F
:10719A00434C4B202D20312020202000436F727257
:1071AA00465245512E2051554152545A0020487A90
:1071BA000020436F72722E20536869667420435709
:1071CA002000487A202020202000436F72722E4629
:1071DA00696C7465722073697A6500436F72722EE6
:1071EA0020535F4C4556454C202D3F0020205049E6
:1071FA004E204130203D2000302042616C6C203D01
:10720A00204F46462056464F2000332042616C6C80
:10721A003D20302E38206D6B562000362042616C9E
:10722A006C3D2036206D6B562020200039204261AB
:10723A006C6C3D203530206D6B56202000392B3286
:10724A003064423D20353030206D6B562000392B9A
:10725A00343064423D2035303030206D6B56003971
:10726A002B363064423D2035303030306D6B56005D
:10727A00535752202020202020503D3057202020D4
:10728A002020005357523D0020503D005720202017
:10729A0000FFFFFFFFFFFFFFFF072B363000FFFF56
:1072AA00FFFFFFFFFFFF072B353500FFFFFFFFFF43
:1072BA00FFFFFF072B353000FFFFFFFFFFFFFFFF38
:1072CA00072B343500FFFFFFFFFFFFFFFF072B34BB
:1072DA003000FFFFFFFFFFFFFFFF072B333500FFE3
:1072EA00FFFFFFFFFFFFFF072B333000FFFFFFFF0A
:1072FA00FFFFFFFF072B323500FFFFFFFFFFFFFFF6
:10730A00FF072B323000FFFFFFFFFFFFFFFF072BB6
:10731A00313500FFFFFFFFFFFFFFFF072B31300072
:10732A00FFFFFFFFFFFFFFFF072B352000FFFFFFD7
:10733A00FFFFFFFFFF0720202000FFFFFFFFFFFFE7
:10734A00FF062020202000FFFFFFFFFFFF0520206F
:10735A0020202000FFFFFFFFFF0420202020202004
:10736A0000FFFFFFFF032020202020202000FFFF36
:10737A00FF02202020202020202000FFFF012020C3
:10738A002020202020202000FFFF20202020202055
:10739A002020202000FF2020202020202020202024
:1073AA002000202020202020202020202020004CE7
:0A73BA0000555342004641003B001D
:00000001FF
